:020000040000fa
:080000000002040000000000f2
:020000040000fa
:100008009a0200009a0200009a0200009a02000078
:100018009a0200009a0200009a0200009a02000068
:100028009a0200009a0200009a0200009a02000058
:100038009a0200009a0200009a0200009a02000048
:020000040000fa
:020000040000fa
:100400002fe220000eff27000e01880000000000f0
:10041000000020000000e000020032000001200087
:10042000200288000c000700004627000100200081
:1004300011000700000020000000e0000200320070
:1004400000000200000000004473020000000000f1
:100450000040da000000fe004440a900a025200072
:100460000000e0000300320000002000a00188002e
:100470004440a80000000600910188008000780038
:100480000000eb0015003700e280400032a0b4000d
:100490009101ba00e280400032a0b4009102ba009b
:1004a000e280400032a0b4000002eb00472bde00e7
:1004b000f507b200602ce10004003a000059eb009f
:1004c0008301e900fdff3e00040037006128e100e0
:1004d000010032000082eb00040007001101ba00a5
:1004e0000200e000e8ff3a00000006003159ba00bf
:1004f0008301e9000c0032002159ba008301e900b0
:10050000080032000400e00003003a00e2804000ee
:1005100032a0b400f5ff370011d9ba008301e90019
:10052000faff3a008100e800e180400032a0b40008
:10053000000006000040da000000fe0080007800a5
:100540001104b100030035009101b10001003c002d
:100550000050a00000000600800078001106b100e5
:10056000030035009101b10001003c000050a100e2
:10057000000006006022b800060220000000d00043
:100580008180d2000482d2008582d2000000a000c7
:100590000202520083825a0003003100020242002c
:1005a00083824a000000a1000603e900f3ff3a003d
:1005b00000000600800178000200370081597800b1
:1005c0000201e9000200e000fcff3a000000060022
:1005d0000001780002007800b041780081cf51001e
:1005e000030032000304e000f9ff3a000001eb00d1
:1005f000020078000000060000017800b141780098
:10060000035978000304e000fcff3a0000000600f4
:10061000800078003104e000feff3a000080ea002c
:1006200000804000000006008001780006003700ce
:100630000201e900b1427800855978000302780090
:100640000504e00006003200030278000200e0002a
:10065000f7ff3a0002003700005aeb000201e90000
:0c0660000200e000fcff3a000000060071
:020000040000fa
:10066c00010000000000000001000000000000007c
:10067c00010000000000000001000000000000006c
:10068c00010000000000000001000000000000005c
:10069c00010000000000000001000000000000004c
:1006ac00010000000000000001000000000000003c
:1006bc00010000000000000001000000000000002c
:1006cc00010000000000000000000000000000001d
:1006dc00010000000000000001000000000000000c
:1006ec0001000000000000000100000000000000fc
:1006fc0001000000000000000000000000000000ed
:10070c0000000000000000000100000000000000dc
:10071c0001000000000000000100000000000000cb
:10072c0001000000000000000000000000000000bc
:10073c0000000000000000000000000000000000ad
:10074c00010000000000000001000000000000009b
:10075c00010000000000000000000000000000008c
:10076c00000000000000000000000000000000007d
:10077c00000000000000000001000000000000006c
:10078c00010000000000000000000000000000005c
:10079c00000000000000000000000000000000004d
:1007ac00000000000000000000000000000000003d
:1007bc00010000000000000000000000000000002c
:1007cc00000000000000000000000000000000001d
:1007dc00000000000000000000000000000000000d
:1007ec0000000000000000000000000000000000fd
:1007fc0000000000000000000000000000000000ed
:10080c0000000000000000000000000000000000dc
:10081c0000000000000000000000000000000000cc
:10082c0001000000000000000100000000000000ba
:10083c0001000000000000000100000000000000aa
:10084c00010000000000000001000000000000009a
:10085c00010000000000000001000000000000008a
:10086c00010000000000000001000000000000007a
:10087c00010000000000000001000000000000006a
:10088c00010000000000000000000000000000005b
:10089c00010000000000000001000000000000004a
:1008ac00010000000000000001000000000000003a
:1008bc00010000000000000000000000000000002b
:1008cc00000000000000000001000000000000001b
:1008dc00010000000000000001000000000000000a
:1008ec0001000000000000000000000000000000fb
:1008fc0000000000000000000000000000000000ec
:10090c0001000000000000000100000000000000d9
:10091c0001000000000000000000000000000000ca
:10092c0000000000000000000000000000000000bb
:10093c0000000000000000000100000000000000aa
:10094c00010000000000000000000000000000009a
:10095c00000000000000000000000000000000008b
:10096c00000000000000000000000000000000007b
:10097c00010000000000000000000000000000006a
:10098c00000000000000000000000000000000005b
:10099c00000000000000000000000000000000004b
:1009ac00000000000000000000000000000000003b
:1009bc00000000000000000000000000000000002b
:1009cc00000000000000000000000000000000001b
:1009dc00000000000000000000000000000000000b
:1009ec0000950000000000000000000001f900006c
:1009fc000000000000000000088700000400000058
:100a0c000000000009af0000000000000100000021
:100a1c000a1b000000000000010000000cc30000d5
:100a2c0000000000000000000daf000002000000fc
:100a3c000000000010ff000000000000000000009b
:100a4c0011ff0000000000000100000012ff000078
:100a5c00000000000100000018ff00000000000072
:100a6c000100000019ff0000000000000100000060
:100a7c0020ff0000000000000000000021ff00002b
:100a8c00000000000000000026df00000100000054
:100a9c0000000000377300000000000000000000a0
:100aac003a25000004000000000000003b25000077
:100abc0000000000000000007200000007000000b1
:100acc00000000000600000000000000050000000f
:100adc000000000004000000000000000300000003
:100aec0000000000020000000000000001000000f7
:100afc0000000000000000000000000007000000e3
:100b0c000000000007000000000000002e2e000076
:040b1c0000000000d5
:020000040000fa
:100b20000200fa000000eb00000f7800050037001b
:100b300020ce20001e00400011c0b3000148780004
:100b40001e0fe8001e007800e20f5000f8ff34008e
:100b50001e68ef001868ef000080eb008080eb005b
:100b600060418800714188000080eb008080eb00cc
:100b700080418800914188002131070080d8200001
:100b80003d0207000004e00033003a00a04180006d
:100b900081d8200001087800a04180008000eb008f
:100ba00051009800a04180008000eb006100980097
:100bb000a24180006000b80070019800010998000f
:100bc000a24180006000b800100998002109980037
:100bd000a0418000c1c5b30041589800100020001a
:100be000000f780006003700a04180001e00400082
:100bf0007c00400001c2b300014878001e0fe800ed
:100c00001e007800ea0f5000f7ff3400a04180007a
:100c10008000eb0041109800a041800001012000fd
:100c200061109800a24180000041800011418000c5
:100c30007011980001199800a241800000418000c5
:100c40001141800010199800211998002468ef00c4
:100c500010002000010037000000eb000080fa00c7
:100c6000000006001400fa00881f78007007980042
:100c7000010f980022579800335798007e0090008b
:100c80004010900060079800b00020001007980006
:100c90007e00900080189000701090007e019000ff
:100ca00010199800211998000e089000601190000a
:100cb000020078000080ea008180ea0020079800a6
:100cc0006e0090000000e0000a003a006c0047004f
:100cd00012c0b300800078007e0090007407070007
:100ce0000000e00010003a00b0012000100798005a
:100cf0000d0037006e0090006f0060000000e00003
:100d0000090032006c00470012c0b3008000780078
:100d10007e009000660707000000e00002003a0035
:100d2000b0012000100798001e009000fb0f50003b
:100d3000c10032001e0090000000e000bb00320045
:100d40006c004700800078007e0090009b0b07003d
:100d5000604798006e409000e24f5000b5003200ae
:100d60006e4090000004e0009d003a007e0090007c
:100d7000e010900041079800ce009000f0032000a2
:100d800000806000400798003e5090000080fb000b
:100d90000000e00003003200e10f500028003200a4
:100da0009e0037004e009000e80f50009200320085
:100db0000000eb0010079800d0c6b300204f980049
:100dc0000040eb00004f7800190037001e80fb0048
:100dd000fe0090007c00400061407800204f9800a9
:100de0001e80fb008e0890007c004000614078006f
:100df000304f98002e4890000080fb00cffd070088
:100e0000000478003e4890000080fb00cbfd070006
:100e1000800f540005003200b00020001007980039
:100e200000000000000000007c0037001e4fe800ba
:100e30001e407800ea4f5000e4ff3600770037008c
:100e4000ce0090002e009000008060000000e000c6
:100e50006b003a004e009000ef0f50006a00320025
:100e60000000eb0010079800d0c6b300204f980098
:100e70000e089000c0589000a0c2b30080cf500070
:100e8000270032000040eb00004f78001f003700c1
:100e90001e80fb00fe0090007c0040006140780056
:100ea000204f98001e80fb008e0890007c004000c0
:100eb00061407800304f9800be489000a0c2b30057
:100ec00080cf500015003200be489000f0c3b30040
:100ed00080cf50000c0032002e4890000080fb00b4
:100ee00096fd0700000478003e4890000080fb005b
:100ef00092fd0700800f540003003200b000200074
:100f000010079800060037001e4fe8001e407800ca
:100f1000e74f5000deff3600010037000000000000
:100f20000e089000c0609000a0c2b30080cf5000b7
:100f3000370032001e0090000000e00036003a004a
:100f400080c0b300004f7800200037001e80fb00f7
:100f5000fe0090007c00400061407800204f980027
:100f60001e80fb008e0890007c00400061407800ed
:100f7000304f9800be489000a0c2b30080cf500010
:100f800001003a0015003700be489000f0c3b300de
:100f900080cf50000c0032002e4890000080fb00f3
:100fa00066fd0700000478003e4890000080fb00ca
:100fb00062fd0700800f540003003200b0002000e3
:100fc00010079800050037001e4fe8001e4078000b
:100fd000ea4f5000ddff3600100037000f003700e9
:100fe0002e5090000004e0000c003a000000eb00de
:100ff00010079800090037000000000007003700c4
:10100000000000000500370000000000030037006a
:101010000000000001003700000000006e0090009a
:101020000000e8006007980042ff37000000000061
:1010300001003700000000001e0090004f047800ff
:101040000080fa00000006001000fa005007980027
:1010500061079800624f98000000eb00000f7800d5
:101060005e00900090007800110798001e0090002c
:10107000306090000004e00003003a00700020009f
:10108000000f7800890037005e0090008018900003
:10109000701090005e0190001019980021199800be
:1010a0006e009000100078000000e00009003a0097
:1010b00012c0b300ee0090005e0090007c060700b6
:1010c0000000e00010003a00b0012000000f78009e
:1010d0000d0037006e009000100078006f00600077
:1010e0000000e0000800320012c0b300ee009000e3
:1010f0005e0090006e0607000000e00002003a006b
:10110000b0012000000f7800ee0090005e0090001b
:10111000aa0a0700404798004e4090000004e000f3
:1011200003003200b0002000000f78005f0037009d
:101130005e0190006000b8007001980001099800fd
:101140005e009000a0009000100090005e019000f2
:1011500030019800410198005e0090008000eb0093
:10116000510098005e0090008000eb006100980044
:101170004e409000e14f500003003a00b0002000c4
:10118000000f78002c0037005e009000c000900037
:10119000300090000001be001e009000d70f070035
:1011a00030079800410798001cc8bf000004e00009
:1011b00005003200e61107000004e00002003200e2
:1011c000900020003a0037005e019000d240880075
:1011d00082418000934180003e009000ce0090004c
:1011e000800f5100818f5900130032001e68ef00fc
:1011f0001e0090009080fb00104090000080fb00db
:101200004800dd0000807000000178003e00900082
:10121000ce009000593007000004e00002003a00c0
:1012200080002000000f78003e019000ce01900069
:101230008241880093418800de00900031089000d0
:101240000020a100b0089800ee48900070c7b300dd
:1012500080cf500004003200ee48900010c6b3006a
:1012600080cf500009003a00de0090003108900065
:101270000000a000b0089800de0090003108900047
:101280000010a100b008980008003700de009000b0
:10129000310890000000a100b0089800de00900026
:1012a000310890000010a000b00898001e007800df
:1012b0000080fa00000006001a00fa00200f9800d3
:1012c000320f9800430f98000040eb00004f980049
:1012d0002e08900090007800510798005e00900062
:1012e000206090000080fb00e10f50000a003200f7
:1012f000e30f500010003a0080ff2f00f1ff2000a4
:101300002007980031079800f0ff2f00f1ff200020
:10131000008fbe001000370080ff20000100200079
:101320002007980031079800f0ff2f0001002000ef
:10133000008fbe000800370080ff2f000100200052
:101340002007980031079800f0ff2f0001002000cf
:10135000008fbe00000000002e08900030019000b9
:10136000c001900062079800730798006e0190001a
:10137000fe0190005e009000a4150700000f980089
:10138000110f98000e0890009e089000be0f5000ac
:10139000ae8f580003003a0080c0b300004f9800a1
:1013a0001f0037005e019000c25190008381fb0056
:1013b000525290000482fb004822dd0084817100bb
:1013c00003007800e25190008381fb00725190008d
:1013d0000281fb004811dd0002817100820078006b
:1013e0000e0990009e099000820f5000838f5800d4
:1013f00002003e00a0c0b300004f98000e0990000c
:101400009e0990002e009000be009000800f5100b9
:10141000818f590002003900c0c3b300004f98000b
:101420002e0890000e0990009e099000320098004e
:10143000430098003e089000ce08900061005000e4
:10144000e0805800300f9800410f98003e0890004f
:10145000ce089000e00f5000e08f580003003200eb
:101460000e4890000004e000bbff32000e489000e0
:101470000080fa00000006000600fa00200798002d
:101480000040eb00004f78002e0090008040eb0001
:10149000316098002e00900001842000f20f20009f
:1014a0000281600090417800e0c1610002c17100da
:1014b00002487800c808de001041900060416100d9
:1014c0008140710011409800013107001007980019
:1014d0001e009000104078000004e000050032007b
:1014e00060c0b300004f780060c0b30024e8b700cc
:1014f0003a0037001e009000900078000010200095
:10150000008060000000e000250032001e00900016
:10151000100090006101b8002e009000f10f200033
:1015200081006100005a90006042620081407200b8
:1015300001589800c810de00105a90006042620006
:101540008140720011589800f10f200081806100e5
:10155000205a900060426200814072002158980039
:10156000c818de0030599000604161008140710070
:10157000315898001e00900090009000002020003c
:10158000808f50000600360010c2b300004f780074
:1015900010c2b30024e8b7001e40780010003700e6
:1015a0002e00900010000700004f78001e407800c9
:1015b0000004e00009003a002e009000240107001a
:1015c000004f78001e4078000004e00003003a005d
:1015d0002e00900011c0b300316098001e407800ca
:1015e0000080fa00000006000a00fa004007980098
:1015f0000040eb00004f78004e0090009080fb0010
:10160000104090000080fb004800dd00008070006a
:10161000000178006000b800582f0700e14f50002b
:101620000500320080c0b300004f780080c0b300d6
:1016300024e8b700030137004e0090009080fb00c3
:10164000104090000080fb004800dd00008070002a
:10165000100798001e009000e0f8930050c5b300fa
:1016600080cf500097003a001e009000f0f89300e1
:10167000a0cab30080cf500092003a004e00900004
:101680009080fb00104090000080fb004800dd00cf
:101690000080700061032000530e070061c4b30096
:1016a000814f50003e003a004e0090009080fb00b9
:1016b000104090000080fb004800dd0000807000ba
:1016c00071032000480e070011c4b300814f500081
:1016d00033003a004e0090009080fb0010409000d4
:1016e0000080fb004800dd000080700081032000c6
:1016f0003d0e070041c5b300814f500028003a005d
:101700004e0090009080fb00104090000080fb0095
:101710004800dd000080700091032000320e0700b9
:1017200011c3b300814f50001d003a004e009000dd
:101730009080fb00104090000080fb004800dd001e
:101740000080700061022000270e070091c2b300e4
:10175000814f500012003a004e009000a0409000cf
:10176000e0c0600021409800b0409000e0c0600000
:1017700031409800c0409000e0c0600041409800b7
:10178000d0409000e0c06000514098004e009000b2
:1017900021c0b300216098000040eb00aa00370090
:1017a0004e0090009080fb00104090000080fb00f5
:1017b0004800dd0000807000210520000a0e0700af
:1017c00061c4b300814f50003e003a004e009000cb
:1017d0009080fb00104090000080fb004800dd007e
:1017e0000080700031052000ff0d070011c4b30018
:1017f000814f500033003a004e0090009080fb0073
:10180000104090000080fb004800dd000080700068
:1018100041052000f40d070041c5b300814f500081
:1018200028003a004e0090009080fb00104090008d
:101830000080fb004800dd000080700051052000a2
:10184000e90d070031c3b300814f50001d003a007d
:101850004e0090009080fb00104090000080fb0044
:101860004800dd000080700021042000de0d07002c
:1018700091c2b300814f500012003a004e00900018
:10188000a0409000e0c0600021409800b04090006f
:10189000e0c0600031409800c0409000e0c06000af
:1018a00041409800d0409000e0c060005140980056
:1018b0004e00900031c0b300216098000040eb0062
:1018c000610037004e0090009080fb0010409000b7
:1018d0000080fb004800dd000080700020079800b9
:1018e0002e009000e0f8930050c5b30080cf500068
:1018f00005003a002e009000f0f89300a0cab30053
:1019000080cf50000500320040c0b30024e8b7008b
:1019100040c0b300004f78004a0037002e0090000e
:10192000e0c093008180fb0070c293000482fb0042
:101930004822dd00848070000101780080c8930097
:101940008180fb0010c893000080fb004800dd0090
:1019500000807000800178004e009000f10f2000a0
:10196000810061002042900060426200814072006c
:1019700021409800c810de003042900060426200b2
:101980008140720031409800f10f20008180610099
:1019900040429000604262008140720041409800e5
:1019a000c818de0050419000604161008140710024
:1019b000514098002e009000a0c09300614798000d
:1019c0006e4090000080fb00ee0f500019003e00ba
:1019d000110020000008dd000105240081006000e6
:1019e0000100e0000b003a0001802100810060004e
:1019f0000100e0000b003a00620060000000e0001f
:101a00000c0032004e00900011c0b300216098001d
:101a10000c0037004e00900021c0b30021609800f8
:101a2000080037004e00900031c0b30021609800dc
:101a30000400370050c0b30024e8b70050c0b30022
:101a4000004f78001e4078000080fa000000060079
:101a50001a00fa00889fbe00400f98000040eb007b
:101a6000404798000000eb00300798000000eb00b2
:101a7000400798004e0890009080fb0010409000b6
:101a80000080fb004800dd000080700080017800cd
:101a90004e099000224290000482fb00b242900066
:101aa0008582fb00c82add00050272000400780070
:101ab000424290000482fb00524190000281fb00f0
:101ac0004811dd00020172008200780003017800f5
:101ad0002a2e0700e14f50000300320080c0b300ff
:101ae00040479800eb0237004e0890009080fb00c2
:101af000104090000080fb004800dd000080700076
:101b0000500798005e009000e0f8930050c5b300c5
:101b100080cf500005003a005e009000f0f893007e
:101b2000a0cab30080cf50000300320030c0b30021
:101b3000404798001b0237004e0890009080fb0041
:101b4000104090000080fb004800dd000080700025
:101b5000e10020002c0d0700600798004e0890005f
:101b60009080fb00104090000080fb004800dd00ea
:101b700000807000d10020001b0d0700ce089000ef
:101b8000906098004e099000a24190008381fb0074
:101b9000324290000482fb004822dd008481710003
:101ba00003007800c24190008381fb005241900005
:101bb0000281fb004811dd00028171008200780083
:101bc0006e0190008001eb0000014100818149001d
:101bd0004e089000f10f20008100610060429000eb
:101be000604262008140720061409800c810de00cf
:101bf0007042900060426200814072007140980023
:101c0000f10f200081806100004a90006042620074
:101c10008140720001489800c818de001049900009
:101c20006041610081407100114898004e089000a9
:101c30009080fb00104090000080fb004800dd0019
:101c40000080700001012000e70c0700ce08900022
:101c5000806098004e0890009080fb00104090003b
:101c60000080fb004800dd00008070006101200062
:101c7000e50c07006101b8004e089000f10f20004c
:101c800081006100405a9000604262008140720011
:101c900041589800c810de00505a9000604262001f
:101ca0008140720051589800f10f2000818061003e
:101cb000605a900060426200814072006158980052
:101cc000c818de00705990006041610081407100c9
:101cd000715898004e099000c25990008381fb0012
:101ce000525a90000482fb004822dd00848171007a
:101cf00003007800e25990008381fb007259900044
:101d00000281fb004811dd00028171008200780031
:101d1000e00f5000e08f580020003a004e0890007d
:101d20009080fb00104090000080fb004800dd0028
:101d30000080700041022000cd0c07000001be00b1
:101d40004e089000f10f200081006100405a900081
:101d5000604262008140720041589800c810de0065
:101d6000505a9000604262008140720051589800c1
:101d7000f10f200081806100605a90006042620093
:101d80008140720061589800c818de0070599000b8
:101d90006041610081407100715898004e089000c8
:101da000e04090008180fb00704190000281fb00c8
:101db0004811dd00828070000102780080489000a8
:101dc0008180fb00104890000080fb004800dd008f
:101dd00000807000800278004e0890000060900043
:101de0000081fb008001eb004e0b9000c65b900071
:101df0008783fb00565c90000884fb004844dd00ac
:101e00008883730007007800e65b90008783fb00ff
:101e1000765b90000683fb004833dd000683730089
:101e200086007800009bb90006037800028cb90098
:101e300088037800070343000010b8000103430043
:101e40008600780004014000858148004e0890001b
:101e5000f10f200081006100204a90006042620082
:101e60008140720021489800c810de00304a90007e
:101e7000604262008140720031489800f10f2000fa
:101e800081806100404a900060426200814072009f
:101e900041489800c818de00504990006041610038
:101ea00081407100514898004e0890009080fb00de
:101eb000104090000080fb004800dd0000807000b2
:101ec00011012000500c0700800078004e0890009f
:101ed000f20f200002816000a0519000e0c161007b
:101ee00002c1710022509800c808de0030519000f5
:101ef0006041610081407100315098004e089000af
:101f00009080fb00104090000080fb004800dd0046
:101f100000807000310120003b0c07008000eb00c6
:101f2000008fbe001e00be00e00f5000e08f580082
:101f300009003a004e0890009080fb00104090008d
:101f40000080fb004800dd000080700001022000de
:101f5000470c0700008fbe004e0890009080fb00e9
:101f6000104090000080fb004800dd000080700001
:101f7000b1002000240c0700700798007e0090003c
:101f80000000e000050032007e009000610060006b
:101f9000004078000004e0000300320010c2b300eb
:101fa00040479800ff0037004e089000a050900076
:101fb0008180fb00305090000080fb004800dd0075
:101fc00000807000c500dd007e00900000804000b1
:101fd0008000e9007e0090000001780011000900f7
:101fe0008280d8008000eb00000f9800110f98004d
:101ff0006e0090006103b8004e08900000609000f1
:102000000081fb008001eb004e0a9000c45a900052
:102010008582fb00545c90000884fb004844dd008e
:102020008882720005007800e45a90008582fb00e7
:10203000745a90000482fb004822dd000482720082
:1020400084007800009ab90004027800028cb9007c
:1020500088027800050242000010b8000102420028
:102060008400780006014000878148000e08900037
:102070009e08900002004000838048003e0110004e
:10208000ae8118000200be00200f9800310f9800aa
:102090004e089000106090000080fb008000eb0074
:1020a0000001be002e089000be08900031f9070024
:1020b0000001be004e089000f10f20008100610079
:1020c000405290006042620081407200415098008e
:1020d000c810de00505290006042620081407200e1
:1020e00051509800f10f20008180610060529000f3
:1020f000604262008140720061509800c818de00a2
:1021000070519000604161008140710071509800f1
:102110004e099000c25190008381fb005252900002
:102120000482fb004822dd008481710003007800f6
:10213000e25190008381fb00725190000281fb000c
:102140004811dd00028171008200780042ff20000a
:1021500003002000820f5000838f580004003e00cf
:102160004e08900011c0b300216098001b0037009a
:102170004e099000c25190008381fb0052529000a2
:102180000482fb004822dd00848171000300780096
:10219000e25190008381fb00725190000281fb00ac
:1021a0004811dd00028171008200780042ff2f009b
:1021b00003002000820f5000838f580004003e006f
:1021c0004e08900021c0b300216098000300370042
:1021d0004e08900031c0b300216098004e08900076
:1021e00020609000e34f500035003a004e08900008
:1021f0009080fb00104090000080fb004800dd0054
:1022000000807000c1022000990b07000041880087
:10221000114188004e099000a24990008381fb0083
:10222000324a90000482fb004822dd008481710064
:1022300003007800c24990008381fb00524990005e
:102240000281fb004811dd000281710082007800ec
:102250000e0990009e099000000141008181490013
:102260004e089000f10f200081006100604a90004c
:10227000604262008140720061489800c810de0030
:10228000704a90006042620081407200714898007c
:10229000f10f2000818061000052900060426200d6
:1022a0008140720001509800c818de001051900063
:1022b0006041610081407100115098003300370087
:1022c0002028ef002228ef004e099000a24990003c
:1022d0008381fb00324a90000482fb004822dd002b
:1022e0008481710003007800c24990008381fb0063
:1022f000524990000281fb004811dd00028171000b
:10230000820078004e099000a25190008381fb006a
:10231000325190000281fb004811dd000281710002
:102320004411de008001eb00000141008181490081
:102330004e089000f10f200081006100604a90007b
:10234000604262008140720061489800c810de005f
:10235000704a9000604262008140720071489800ab
:10236000f10f200081806100005290006042620005
:102370008140720001509800c818de001051900092
:10238000604161008140710011509800fe00900092
:1023900000202000808f50000200360010c2b300e1
:1023a000404798004e08900020609000e34f500096
:1023b0000d0032004e4090000004e000ae003200fc
:1023c0005e009000a0c0900090c2b30080cf50008b
:1023d000050032005e009000a0c0900080c2b300f3
:1023e00080cf5000a6003a005e009000b0509000f0
:1023f0008180fb00405090000080fb004800dd0021
:10240000008070000000e0003a003a005e0090009a
:10241000407090000004e00036003a005e0090003a
:10242000507090000004e00032003a005e0090001e
:10243000607090000004e0002e003a005e00900002
:10244000707090000004e0002a003a005e009000e6
:10245000007890000004e00026003a005e00900042
:10246000107890000004e00022003a005e00900026
:10247000207890000004e0001e003a005e0090000a
:10248000307890000004e0001a003a005e009000ee
:10249000407890000004e00016003a005e009000d2
:1024a000507890000004e00012003a005e009000b6
:1024b000607890000004e0000e003a005e0090009a
:1024c000707890000004e0000a003a005e0090007e
:1024d000a0c0900090c2b30080cf5000070032002f
:1024e0005e009000a0c0900080c2b30080cf50007a
:1024f0000200320030c0b300404798004e409000c8
:102500000004e000300032003e0090000000e000d7
:102510002d003a0010002000300798004e0890006f
:102520009080fb00104090000080fb004800dd0020
:1025300000807000000278004e099000a2419000d7
:102540008381fb00b24290008582fb00c82add0037
:102550008581710003007800c24190008381fb00f7
:10256000524190000281fb004811dd0002817100a0
:10257000820078005e019000a27190008381fb00d0
:10258000327190000281fb004811dd000281710070
:102590008001eb00000041008180490004017800c7
:1025a000762b0700e14f50000400320080c0b300da
:1025b00024e8b70080c0b3003d0037000040eb00c6
:1025c000404798002b0037004e4090000004e00088
:1025d0002d0032004e0090000000e0002c003a0078
:1025e00010002000400798004e0890009080fb00eb
:1025f000104090000080fb004800dd00008070006b
:10260000800178004e099000224290000482fb0075
:10261000b24290008582fb00c82add0005027200ec
:1026200004007800424290000482fb005241900076
:102630000281fb004811dd00020172008200780077
:1026400066004000e0804800030178004b2b070043
:10265000e14f50000400320080c0b30024e8b7000e
:1026600080c0b300120037000040eb0040479800e4
:102670000000000023fd37000000000005003700c7
:1026800000000000030037000000000001003700d8
:10269000000000004e4090000004e0000300320003
:1026a000ce40900043822000814978004e40900047
:1026b0004f04be000080fa00000006000600fa0089
:1026c000200798006000b800008fbe002e00900028
:1026d000200890008000eb00008fbe001e00be00ae
:1026e000c000dd0000002000008fbe002e00900022
:1026f000500890008000eb001e1f70001e977000b5
:102700001e00be000080fa00000006001000fa0063
:1027100060079800710798006e00900090007800a4
:10272000110798006e00900010199000a0199000f9
:1027300022079800330798007e0090001000780070
:102740006102b8001e019000825990008381fb0055
:10275000125b90000683fb004833dd008681710028
:1027600003007800a25990008381fb003259900049
:102770000281fb004811dd000281710082007800b7
:10278000cb09dd004500de0000807100c508de00d9
:102790000001be000400be0076f707001047980055
:1027a0001e009000206090000080fb00e10f5000b0
:1027b00022003500e20f50000d003400e30f5000fe
:1027c0001e003a001e009000106090009e40900095
:1027d0008180fb000080fb000001780011000900ef
:1027e0008280d8008000fd00104798001300370059
:1027f00000418000114180002e019000be01900038
:10280000800f5100818f59000b0032001e00900094
:10281000106090009e4090008180fb000080fb00d3
:1028200080017800110009008380d8008000fd003d
:102830001047980001003700000000002e019000b2
:10284000be0190001e0090002c0a0700400798006f
:10285000510798001e0090009080fb0010409000ef
:102860000080fb004800dd0000807000000278005e
:102870001e4090000081fb008001eb004e009000a4
:10288000de00900002004000838048008041eb00a1
:1028900004017800302b07000004e00003003a0038
:1028a0000040eb00004f78000200370010c0b3007a
:1028b000004f78001e4078000080fa0000000600fb
:1028c0001400fa0070079800010f9800120f98008a
:1028d0000000eb00400798001e0890002060900068
:1028e0000080fb00e10f50000a003200e30f5000af
:1028f00010003a00f0ff2f00f1ff200020079800a1
:102900003107980080ff2f00f1ff2000008fbe00ec
:1029100010003700f0ff2f00010020002007980072
:102920003107980080ff200001002000008fbe00ca
:1029300008003700f0ff2f0001002000200798005a
:102940003107980080ff2f0001002000008fbe009b
:10295000000000007e0090008e089000e00f500004
:10296000e08f5800070032007e0190008e09900031
:102970001000200001002000800f5100818f5900bd
:102980003b003a0020002000400798003b00370041
:102990007e0190008e0990001e0890001b10070019
:1029a00050079800610798005e019000ee019000ca
:1029b0002e009000be009000800f5100818f5900c2
:1029c00003003a001000200040079800280037005c
:1029d0005e009000ee009000e00f5000e08f580085
:1029e000070032005e019000ee0190001000200010
:1029f00001002000800f5100818f590003003a0030
:102a00002000200040079800190037005e00900069
:102a1000ee009000be0f5000ae8f5800020039004b
:102a200020002000400798008040eb006022b800a2
:102a30007e0190008e0990001e089000fa11070098
:102a40000001be002e009000be009000800f5100db
:102a5000818f590002003a001000200040079800c2
:102a60005e019000ee01900072079800030f98003d
:102a70004e0090000000e000c5ff320011c0b3001e
:102a80006022b8006011b8001e089000e61107002f
:102a90004e009000e20f500002003a0010c0b30058
:102aa000010037000040eb000080fa000000060043
:102ab0001c00fa00300f9800410f9800225f980028
:102ac0003e08900090007800610798003e08900052
:102ad000701190008019900072079800030f980001
:102ae0003e08900010199000a0199000320798003d
:102af000430798004e089000100078006102b8006b
:102b00006e019000825990008381fb00125b90005f
:102b10000683fb004833dd008681710003007800e6
:102b2000a25990008381fb00325990000281fb0082
:102b30004811dd000281710082007800cb09dd00c0
:102b40004500de0000807100c508de000001be0007
:102b50000400be0087f60700204f98006e0090002a
:102b6000206090000080fb00e30f50000f003a004f
:102b70006e00900010609000ae4890008180fb00d5
:102b80000080fb0000017800110009008280d8005d
:102b90008000fd00204f980080ff2f00f1ff2000f3
:102ba0001007980021079800140037007e0090005d
:102bb0008e089000e00f5000e08f58000a003200ad
:102bc0006e00900010609000ae4890008180fb0085
:102bd0000080fb0080017800110009008380d8008c
:102be0008000fd00204f980080ff2f000100200092
:102bf0001007980021079800000000002e58900050
:102c00000004e00005003a004e0890001000780033
:102c10006f0060000000e000b2003a002e48900013
:102c20000004e00004003a004e0890001000780014
:102c3000ef0f500003003e002e5890000004e0000b
:102c40002f0032007e0090008e089000e00f5000b0
:102c5000e08f580004003a006000b8003007980088
:102c600041079800260037002e5890000004e0002d
:102c70000b0032004e089000900078006e0090002b
:102c8000106090000080fb004400dd00000178002f
:102c9000110009008280d800304f980013003700df
:102ca00010c0b300304f9800100037003e01900074
:102cb000ce0190006e009000540f0700300798007e
:102cc000410798003e019000ce0190001e00900048
:102cd000ae009000800f5100818f59000700310035
:102ce0003e4890000040e900304f98003e48900078
:102cf0000004e000edff3a00010037000000000092
:102d00003e019000ce0190001e009000ae009000a9
:102d1000800f5100818f59006d0031003e089000f6
:102d20003e019000ce0190001218980023189800e0
:102d30003e019000ce0190006e009000ef08070069
:102d4000100f9800210f9800004180001141800071
:102d50003e019000ce019000800f5100818f5900fc
:102d600020003a002e4890000081fb008001eb001b
:102d70001e089000ae0890000202400083824800c6
:102d80006e019000e24990008381fb00724b90003d
:102d90000683fb004833dd00868171000300780064
:102da000825190008381fb00125190000281fb0050
:102db0004811dd000281710082007800800f52000e
:102dc000818f5a00070039006e009000206090004b
:102dd000e34f5000030032000000eb00000f7800ca
:102de0004c0037001cc8bf000004e00005003200a2
:102df000d70a07000004e000020032000000eb00e8
:102e0000450037001a28ef001e68ef006e009000a2
:102e10009080fb00104090000080fb004800dd0027
:102e200000807000000278002e4890000081fb00b6
:102e30008001eb001e089000ae08900002004000e8
:102e400083804800040178004c290700e14f5000be
:102e5000030032000000eb00000f7800170037007d
:102e60002e5890000004e0000d0032006e0090002b
:102e70009080fb00104090000080fb004800dd00c7
:102e800000807000800078004e08900010007800ec
:102e90006f0060004500dd00008f40000700370034
:102ea0006e0090009080fb00104090000080fb00be
:102eb0004800dd0000807000000f78000080eb000b
:102ec0008080eb008041880091418800110037002c
:102ed00010c0b3001de8b7000000eb00000f780041
:102ee0000c0037006e0090009080fb0010409000b6
:102ef0000080fb004800dd0000807000800078004a
:102f00004e089000100078006f0060004500dd0062
:102f1000008f40001e0078000080fa0000000600cc
:102f20001600fa00000f9800110f98004257980001
:102f30000000eb00100798002468ef000040eb0051
:102f4000004f7800080037001e80fb009e80fb00c9
:102f50000e099000fc804000e2c0780000004700ad
:102f6000414098001e4fe8001e407800ea4f500094
:102f7000f5ff36001e0890008000eb000108780085
:102f80009e0890000e089000570007000004e00023
:102f90000f00320064004700ce5190001e099000df
:102fa000800078000e089000dc0007000080fb0025
:102fb000100798001e0090000000e00006003a0094
:102fc0000e0890000a000700100798000200370062
:102fd00040012000100798001e009000004078007b
:102fe00024e8b7001e0090000080fa0000000600f0
:102ff0001000fa00700798007e00900040109000ca
:103000006007980068004700800078007e0090000c
:1030100056070700000f78001e0078000000e0004f
:103020002e003a006c004700800078007e0090007f
:1030300090030700100798004e009000de009000fb
:10304000800078001e009000510898004e0190000a
:10305000de01900000002000f1ff20000202780055
:10306000030178008001780001007800030262000b
:10307000000061008000eb00c000dd0000002000c7
:103080000001be006120b800000171008181710063
:1030900022079800330798002e009000be00900091
:1030a0004008de000100200020079800310798004a
:1030b000ae0090001e009000210898006c004700b0
:1030c000800078007e00900090fd0700e14f5000e6
:1030d0000200320090002000000f78001e007800ef
:1030e0000080fa00000006001000fa006007980057
:1030f0007107980010c0b300004f78006e00900078
:1031000080189000701090006e01900010199800c7
:103110002119980012c0b300fe0090006e009000cc
:1031200063fe0700300798003e0090000000e000ba
:103130006c003a00b0c1b300004f78006f00370058
:103140000040eb00104798007e009000900078004f
:10315000210798000041eb00fe0090006e009000f7
:1031600053fe0700300798003e0090000000e0008a
:10317000030032003e009000104078002047980085
:103180007e009000100078008000e8007e00900033
:10319000010878002e409000fb4f400003003200f1
:1031a0002e4090000004e00009003a003e0090002c
:1031b0000000e000060032001e4090000040e800e1
:1031c000104798001e4090000004e000e1ff32002c
:1031d0003e0090000000e0003a003a006e009000cf
:1031e00010199000a019900042079800530798000a
:1031f00000418000114180004e019000de019000ee
:10320000800f5100818f59001b003a006e00900022
:103210001000780020609000e34f5000030032005f
:1032200020c0b300004f78002e0037006e009000e1
:103230004e019000de01900032009800430098009b
:1032400011c0b3006e00900099000700f54f5000c8
:1032500003003a0020c0b300004f7800210037007f
:103260007e009000ae019000030878000040eb0063
:10327000004f78001b0037006e0090004e01900058
:10328000de019000320098004300980011c0b300a6
:103290006e00900086000700f54f500003003a00d2
:1032a00020c0b300004f78000e0037007e00900071
:1032b000ae019000030878000040eb00004f78005a
:1032c000080037001e409000e14f500005003a0012
:1032d0000040eb00004f78007e009000ae009000b0
:1032e000010878001e407800e14f500094ff320042
:1032f0007e0090002e019000020878001e407800a9
:103300000004e00002003a0010c0b30001003700e2
:103310000040eb000080fa00000006000c00fa00fc
:10332000200798003107980042079800234f980023
:103330000040eb00004f78002e00900080189000b5
:10334000701090002e01900010199800211998001b
:1033500012c0b300ce0090002e009000d4fd0700f4
:10336000100798001e0090000000e00002003a00e4
:10337000b0c1b3004c0037001e009000b200200026
:10338000be009000a8f407002e489000f24f5000b5
:1033900004003a001e00900001c1b30031489800bb
:1033a000030037001e00900001c2b30031489800ae
:1033b0001e0090008040eb00414898001e009000e5
:1033c0008000eb00210898001e0090008000eb00b8
:1033d000510898001e0190006000b8006009980034
:1033e000710998001e00900021cbb300514898004d
:1033f0001e00900081272700710098001e00900099
:10340000012b2300010898001e009000012b2300cf
:10341000110898001e00900091272700310898009d
:103420001e009000012b2300410898001e00900010
:10343000f0089000600890002e019000100998009c
:10344000210998001e009000f00090002e009000ce
:10345000410898001e009000800890002e00900007
:10346000510898001e009000304890008080fb00ba
:103470002e009000611098004e009000900078009f
:103480002e00900041109800ce0090002e00900079
:103490009efc0700e14f50000200320090c0b300d4
:1034a000004f78001e4078000080fa0000000600ff
:1034b0000e00fa0050079800414f98005e009000ff
:1034c000100f78005e00900030019000c001900065
:1034d00012079800230798005e0090004400070040
:1034e00010079800210798001e009000ae00900081
:1034f000e00f5000e08f580002003a0050c1b300c6
:10350000390037001e00780020609000e14f500025
:1035100008003a008040eb0084ff200005002000f6
:103520001e019000ae0190001e0078003e0f0700c3
:10353000130037001e00780020609000e24f50001a
:1035400008003a008040eb0084ff2f0005002000b7
:103550001e019000ae0190001e007800320f07009f
:10356000070037008040eb0084ff2f00f5ff2000ac
:103570001e019000ae0190001e0078002a0f070087
:103580005e00900030019000c0019000320798006a
:10359000430798008040eb001e029000ae029000ae
:1035a0003e019000ce0190001e0078001e0f070023
:1035b0005e0090001e019000ae0190003200980065
:1035c000430098004e489000e14f500005003a003b
:1035d0001e019000ae0190001e0078003b0607001f
:1035e000010037000040eb000080fa0000000600f8
:1035f0001800fa00300f98006000b80060079800cb
:10360000710798003e08900090007800010f980024
:103610003e08900030019000c0019000028fbe0073
:103620000e089000206090000080fb00e10f500029
:103630000b003200e30f500012003a0070ff2f0021
:10364000f1ff20002007980031079800f0ff2f00bd
:10365000f1ff200040079800510798001200370042
:1036600070ff20000100200020079800310798001b
:10367000f0ff2f000100200040079800510798003c
:103680000900370070ff2f0001002000200798007c
:1036900031079800f0ff2f0001002000400798003c
:1036a00051079800000000001e01be00100020001d
:1036b00001002000800f5100818f590003003e005f
:1036c0002000200001002000008fbe001e01be006f
:1036d000120f9800230f98001e01be000e089000e4
:1036e000ca0c07003f0037001e01be000e08900004
:1036f000c60c070060079800710798006e019000e3
:10370000fe0190004e009000de009000800f5100fe
:10371000818f590003003a006000b800008fbe009e
:10372000360037006e009000fe009000e00f500061
:10373000e08f58003000320012002000030020000b
:103740001e0f41005e9749006e019000fe0190003f
:103750002e009000be009000800f5100818f590014
:10376000140032000e099000c25190008381fb00ca
:10377000525290000482fb004822dd0084817100d7
:1037800003007800e25190008381fb0072519000a9
:103790000281fb004811dd00028171008200780087
:1037a00062004000e0804800be0f5000ae8f58001d
:1037b00003003e002000200001002000008fbe001a
:1037c0001e089000ae0890001e01be00800f510040
:1037d000818f590003003a006000b800008fbe00de
:1037e000060037001e00be00e00f5000e08f5800ba
:1037f000bdff3a0001003700000000001e00be00bf
:103800000080fa00000006000a00fa004007980055
:1038100080042000100798002468ef004e009000fc
:1038200040109000300798004e0090003008900043
:10383000610060000000e0004b0032001cc8bf00c7
:103840000004e00007003200410807000004e00027
:103850000400320090c0b30024e8b7000080eb0001
:103860005d0037004e0090001000780011c0b300da
:103870006022b8006011b8006b0e07002c28ef0022
:103880002e28ef004e009000c00090003000900005
:103890004e019000120278000001be000400780082
:1038a0005a0c070066004700800078004e00900028
:1038b00070010700200798002e0090000000e00033
:1038c00006003a00b0c1b30024e8b7000080eb0066
:1038d000100798001e0090003f0037002e00900057
:1038e0003f0007004e009000a008900010089000d4
:1038f0002e01900060099800710998004e00900018
:1039000060109000804078002e00900031489800b0
:1039100066004700800078004e0090007bfb0700a7
:103920000004e000080032006600470080007800d4
:103930004e0090004f010700200798000000eb00a8
:10394000100798000400370090c0b30024e8b700c7
:103950000080eb0010079800ce0090003108900026
:103960000000a100b00898000000eb00000f7800f4
:103970000f0037009e007800600320000088b90027
:103980008000780000c42000808040004e0090003d
:10399000808f500005003a0020ce20001e0040001d
:1039a00011c0b30001487800040037001e0fe80082
:1039b0001e007800e20f5000eeff36009e009000df
:1039c00080042000808f500002003a000000eb00cd
:1039d000100798001e0090000080fa00000006000a
:1039e0000800fa00300798003e0090003008900070
:1039f000004078007f4f60003e009000b0089000cb
:103a0000007e2000008060004500de001047980026
:103a10003e009000300890004b00de0020479800e8
:103a20003e00900040089000004078007f40600019
:103a3000304798003e009000c0089000001e200013
:103a4000008060004500de00404798003e00900086
:103a5000400890004900de00504798001e40780062
:103a6000fc4f500002003e001e4fe8002a003700c5
:103a70000040eb00004f78009e409000a0c3b300d0
:103a800080cf500004003e001e4090000040e8003f
:103a900010479800200037000040eb0010479800c6
:103aa0002e409000f64f500004003e002e40900043
:103ab0000040e80020479800170037000040eb0066
:103ac000204798003e409000fd4f500004003e000b
:103ad0003e4090000040e800304798000e0037005c
:103ae00010c0b300304798004e409000eb4f50009c
:103af00004003e004e4090000040e800404798001f
:103b00000500370010c0b300404798005e409000a9
:103b10000040e800504798009e80fb003e00900067
:103b2000310898003e009000b00890001e409000c0
:103b30000080fb004500dd00810070003e00900029
:103b4000310898003e009000b00890002e40900090
:103b50000080fb004b00dd00810070003e00900003
:103b6000310898003e4090008080fb003e009000ad
:103b7000410898003e009000c00890004e40900020
:103b80000080fb004500dd00810070003e009000d9
:103b9000410898003e009000c00890005e409000f0
:103ba0000080fb004900dd00810070003e009000b5
:103bb000410898000080fa00000006000c00fa009e
:103bc00040079800510798000040eb0040479800dc
:103bd0005e009000100078006f0060000000e000c0
:103be00010003a005e009000100078000000e00035
:103bf0000c0032004e009000801890007010900071
:103c00004e019000101998002119980012c0b300bd
:103c1000de0090004e009000a5fb0700000f78002a
:103c2000050037000041eb00de0090004e009000e0
:103c30009ffb0700000f78001e0078000000e000e6
:103c400003003a0020c0b3003047980086003700d8
:103c50001e00780010407800504798005e409000a9
:103c6000fb4f400003003a0010c0b30030479800fb
:103c70007d0037005e4090000004e00003003a0041
:103c800020c0b30030479800770037001e0078004e
:103c9000b0489000514798000040eb002047980042
:103ca000150037002e4090000080fb009e00780039
:103cb00061407800604798006e4090000080fb00f3
:103cc00025f20700604798004e4090000080fb00fe
:103cd000ee4090004e0190000000410041589800d5
:103ce0004e4090000040e800404798002e40900071
:103cf0000040e800204798002e409000e74f500019
:103d0000e8ff36001e007800b04890005147980048
:103d10001e00780000489000604798000040eb00cb
:103d200020479800160037002e4090000080fb00ce
:103d30009e0078006800400061407800604798006d
:103d40006e4090000080fb0003f20700604798007f
:103d50004e4090000080fb00ee4090004e0190002d
:103d600000004100415898004e4090000040e8009b
:103d7000404798002e4090000040e80020479800ff
:103d80002e409000e24f5000e7ff36005e009000aa
:103d9000900078004e009000411098001e007800be
:103da00010407800504798005e409000fb4f400064
:103db00003003a0010c0b3003047980002003700fb
:103dc0000040eb00304798001e007800f00890009b
:103dd000600890004e019000100998002109980099
:103de0001e00780035fa07004e019000100198007f
:103df000210198001e007800b048900051479800bb
:103e00005e4090008080fb004e00900061109800a2
:103e10005e4090000080fb00700060000000e00049
:103e2000090032001e007800f00090004e00900063
:103e3000410898001e007800800890004e00900015
:103e400051089800080037001e007800b008900064
:103e50004e009000410898001e007800c0089000b5
:103e60004e009000510898003e4090000080fa00fb
:103e7000000006000800fa002007980031079800ab
:103e80002e00900080189000701090002e0190007d
:103e9000101998002119980012c0b300be009000bc
:103ea0002e00900002fb0700000f78001e00780033
:103eb0000000e00002003a000000eb002b00370099
:103ec0001e00780010407800204798002e40900097
:103ed0000004e00002003a000000eb00000f780050
:103ee0001e0078000000e0001f0032002e4090000d
:103ef000fb4f400003003a000000eb00000f780089
:103f0000190037001e007800b04890002147980043
:103f1000120037003e009000100078008000e8009a
:103f20003e009000010878000041eb00be009000c8
:103f30002e009000defa0700000f78001e007800c7
:103f40000000e00002003a000000eb00070037002c
:103f50001e007800b0489000214798002e40900045
:103f6000ef4f5000ebff32001e0078000080fa0097
:103f7000000006001200fa00600798007107980020
:103f8000025798000000eb00000f78006e009000d0
:103f900090007800110798006e009000701190005a
:103fa0008019900022079800330798006e00900057
:103fb0002e019000be01900012189800231898005e
:103fc00012c0b300fe0090006e009000b8fa070027
:103fd000400798004e0090000000e00004003a0006
:103fe00010c0b30024e8b700b00120004100370042
:103ff0004e00900010407800204f98004e00900036
:104000000000e000030032002e4890000004e000b1
:1040100003003a00b0002000000f78002d003700a8
:104020002e489000fb4f400003003a00b0002000f3
:10403000000f7800270037004e009000b049900034
:10404000234f98004e00900051ceb30001487800f5
:104050004e00900099f9070020079800310798005a
:104060001e0078000000e00005003a00fe0090000d
:104070006e009000a5f907000004e00003003a007c
:1040800010002000000f780012003700004180006f
:10409000114180002e019000be019000800f510060
:1040a000818f59000b0032000e5090000004e00098
:1040b000080032001e0190002e009000be0090000b
:1040c000fff907000080fb000000e9004f00de0060
:1040d000000f78001e0078000000e00002003a00a7
:1040e0002468ef000200370010c0b30024e8b700d6
:1040f0001e0078000080fa00000006001800fa0098
:10410000200f9800310f98000040eb0010479800f6
:1041100010002000100f98002468ef003e08900067
:104120000000e00004003a0090c1b30024e8b700aa
:104130000080eb00af0037003e0890007c0040009c
:104140000041eb00800078002e089000480707002f
:104150000004e00004003a0020c1b30024e8b700e6
:104160000080eb00a30037000040eb00004f780018
:10417000080037001e80fb009e80fb003e09900077
:10418000fc804000e2c078000000470061409800d9
:104190001e4fe8001e407800ea4f5000f5ff360041
:1041a0003e089000c0109000110798000000eb003e
:1041b000100f98003e08900080189000701090003a
:1041c0003e099000101998002119980072004700cc
:1041d00012c0b300800078003e08900034fa070057
:1041e000200798002e0090000000e00004003a0034
:1041f000b0c1b30024e8b7000080eb007d003700b9
:104200000040eb00004f78000b0037001e80fb00e1
:10421000ae009000e14078001e80fb0000004700e7
:104220006040900080cf50000200320010c0b30008
:10423000104798001e4fe8001e407800ea4f5000db
:10424000f2ff36001e4090000004e00004003a0037
:1042500010c1b30024e8b7000080eb006500370010
:104260000040eb00104798001d68ef007200470007
:104270000041eb00800078003e0890000cfa070037
:10428000200798002e0090000000e00007003a0090
:104290001dc8bf00e14f500026003200b0c1b3007e
:1042a00024e8b7000080eb00520037002e00900099
:1042b000104078000004e000200032000040eb00d5
:1042c000004f78000b0037001e80fb00ae0090000e
:1042d000e14078001e80fb00000047006040900035
:1042e00080cf50000200320010c0b3001047980089
:1042f0001e4fe8001e407800ea4f5000f2ff3600e3
:104300001e4090000004e00004003a0010c1b30019
:1043100024e8b7000080eb00360037000040eb00d7
:10432000104798001e0890000000e800100f980049
:10433000ceff370000000000010037000000000041
:104340009e009000110f98003e0890008018900089
:10435000701090003e0990001019980021199800e3
:1043600072004700800078003e089000c1fe070000
:10437000200798002e0090000000e00004003a00a2
:10438000b0c1b30024e8b7000080eb00190037008b
:104390000040eb00004f7800080037001e80fb0053
:1043a0009e80fb003e099000fc80400062c17800c6
:1043b000ae009000827078001e4fe8001e4078002a
:1043c000ea4f5000f5ff3600720047008000780089
:1043d0003e089000cdf807000004e00004003a0019
:1043e00090c0b30024e8b7000080eb000100370064
:1043f0000000eb000080fa00000006000e00fa004a
:1044000050079800610798000000eb00000f78004b
:104410000000eb00100798001500370021ce2000a7
:104420001e00900000804000104078000004e00072
:104430000c00320021ce20001e00900000804000c1
:104440008040eb00014878009e009000600320004f
:104450000088b9008000780000c42000008f400070
:10446000060037001e0090000000e80010079800ca
:104470001e009000e20f5000e8ff34001e0078009c
:104480000000e00004003a0000c2b30024e8b700d6
:104490000000eb00930137009e0078007c80400014
:1044a0000041eb00800078005e009000700607007d
:1044b0000004e00009003a0021ce20001e00900018
:1044c0000080400011c0b3000148780020c1b30053
:1044d00024e8b7000000eb00820137006e00900076
:1044e00010407800604798001e00780081d82000b6
:1044f000010878001e0178006000b80010019800e3
:10450000210198001e0178006000b8003001980079
:10451000410198001e0078008000eb0041109800d7
:104520001e0078000102200061109800a041800068
:1045300080189000701090001e0178007011980093
:1045400001199800a0418000a01890001018900058
:104550001e01780010199800211998009e0078001b
:10456000c0d12000e60107008041eb0012c0b3007b
:10457000c1d120001e007800baf107000000e00061
:10458000e1003a006e4090000080fb0071052000c1
:10459000810f50001400320071052000810f50007f
:1045a00007003c0011042000810f5000450032003c
:1045b00021052000810f5000b5003200cd003700ea
:1045c00021072000810f5000b10032007107200048
:1045d000810f50000400320011062000810f5000ae
:1045e00038003200c30037001e00780040109000f1
:1045f000400798006800470012c0b30080007800b0
:104600001e0078005bfe0700200798002e00900037
:104610000000e00004013a00680047000041eb00a0
:10462000800078001e0078003dfa070020079800ff
:104630002e0090000000e000fd003a0068004700f6
:1046400072c7b300800078001e0078007ef2070079
:10465000200798001e007800601090007000600035
:104660000000e00004003200f0c1b30024e8b7000d
:10467000f00f2000200798002e0090000000e000be
:10468000ed003a00210020006011b8001e00780003
:10469000a4070700200798006e0090000000e800c3
:1046a00090407800b0c2b30080cf5000e4003a00e0
:1046b0009e007800310890000010a000b00898001b
:1046c000f40037001e007800a00890001008900049
:1046d000e00f5000e08f5800310032001e007800db
:1046e00040109000400798006800470072c7b30070
:1046f000800078001e00780053f207002007980021
:104700001e00780060109000700060000000e00063
:1047100004003200f0c1b30024e8b700f00f20001d
:10472000200798002e0090000000e000c6003a002c
:10473000210020006011b8001e00780079070700f2
:10474000200798002e0090000000e00003003200d7
:10475000a0c1b30024e8b700060037001e007800af
:10476000c0009000300090000001be0080d8200002
:10477000a60807006e0090000000e8009040780056
:10478000b0c2b30080cf5000b1003a009e00780064
:10479000310890000010a000b0089800bd0037005c
:1047a0001e00780040109000400798006800470005
:1047b00012c0b300800078001e007800edfd0700f5
:1047c000200798002e0090000000e000a2003a00b0
:1047d000680047000041eb00800078001e00780070
:1047e000cff90700200798002e0090000000e0009d
:1047f0009b003a006800470072c7b3008000780051
:104800001e00780010f20700200798001e007800b4
:1048100060109000700060000000e00004003200b2
:10482000f0c1b30024e8b700f00f20002007980083
:104830002e0090000000e0008b003a0021002000d4
:104840006011b8001e0078003607070020079800a6
:104850002e0090000000e00002003200a0c1b30072
:1048600024e8b7006e0090000000e8009040780057
:10487000b0c2b30080cf50007d003a009e007800a7
:10488000310890000010a000b008980081003700a7
:104890001e00780040109000400798006800470014
:1048a00022c7b300800078001e007800e6f1070000
:1048b000200798006e0090000000e800904078000b
:1048c000b0c2b30080cf50006b003a001e007800e9
:1048d00060109000700060000000e00068003a0086
:1048e0009e007800310890000000a000b0089800f9
:1048f00068003700f0c1b30024e8b700f00f2000d3
:104900002007980063003700c1d120001e00780006
:10491000fb000700ee40900070c7b30080cf50004e
:104920000c003200ee40900070c5b30080cf500004
:1049300008003200ee40900010c6b30080cf500057
:1049400004003200ee40900010c4b30080cf50004d
:1049500032003a000000eb00400798006800470072
:104960000041eb00800078001e0078006cf9070021
:10497000200798002e0090000000e00045003a005b
:104980006800470072c7b300800078001e007800fe
:10499000adf10700200798001e007800601090001d
:1049a000700060000000e00004003200f0c1b300bd
:1049b00024e8b700f00f2000200798002e00900098
:1049c0000000e00030003a00210020006011b80033
:1049d0001e007800d3060700200798002e009000e4
:1049e0000000e00002003200a0c1b30024e8b700dc
:1049f0006e0090000000e80090407800b0c2b30064
:104a000080cf500022003a009e00780031089000cc
:104a10000010a000b00898001e003700b000200071
:104a2000200798001b003700000000001900370025
:104a300000000000170037000000000015003700dc
:104a400000000000130037000000000011003700d4
:104a5000000000000f003700000000000d003700cc
:104a6000000000000b0037000000000009003700c4
:104a700000000000070037000000000005003700bc
:104a800000000000030037000000000001003700b4
:104a9000000000002e2307000004e00004003200a4
:104aa0009e007800310890000000a100b008980036
:104ab0002e0090000000e0000800320021ce20000f
:104ac0001e0090000080400011c0b3000148780033
:104ad0000000eb00000f7800010037002468ef00b1
:104ae0001e0078000080fa00000006000200fa00b4
:104af000000f78002468ef001e0078008008900006
:104b0000700090000080fa00000006000600fa0025
:104b10002007980060ce2000000f78002468ef0086
:104b20000b2307000004e0000400320080c1b30042
:104b300024e8b7000080eb00510037009e007800a9
:104b40007c8040000041eb00800078002e00900047
:104b5000c70407000004e00004003a0020c1b300cd
:104b600024e8b7000080eb00450037001e00780005
:104b700081d82000010878001e0178006000b8008c
:104b800010019800210198001e0178006000b80013
:104b900030019800410198001e0078008000eb0071
:104ba000411098001e00780001022000611098005a
:104bb000a041800080189000701090001e017800c5
:104bc0007011980001199800a0418000a018900071
:104bd000101890001e0178001019980021199800f3
:104be0009e007800c0d12000450007008041eb0006
:104bf00012c0b300c1d120001e00780019f00700d8
:104c0000100798001e0090000000e0000400320031
:104c1000b0c0b30024e8b7000080eb0018003700f4
:104c20001e00780060109000700060000000e0003e
:104c30000400320030c1b30024e8b7000080eb006c
:104c40000f003700810220001e80400012c0b30018
:104c5000800078001e007800c6fc0700100798004e
:104c60001e0090000000e00002003a000000eb008f
:104c70000300370010c0b30024e8b7000080eb0049
:104c80000080fa00000006000200fa00000f780021
:104c90001cc8bf000004e000010032002c03070024
:104ca0001e0178006000b8007001980001099800aa
:104cb0001e0078008000eb00610098001e00780064
:104cc0008000eb00510098001e007800a0009000ca
:104cd000100090001e0178003001980041019800fa
:104ce0001a28ef000080fa00000006000000fa0019
:104cf00024c8bf000080fb000080fa00000006000e
:104d00000c00fa004007980051079800ce00900070
:104d100011079800de0090002107980060c3b300df
:104d2000604798000040eb00004f78000900370012
:104d30001e80fb009e009000008040009e80fb00d3
:104d40002e019000810041009140780001487800d8
:104d50001e4fe8006e4090009e40780080cf5000cb
:104d6000f3ff39000080fa00000006000800fa0096
:104d700020079800310798000000eb00000f780032
:104d80002e00900090007800110798002e009000ef
:104d900017fa07003e0190000089be003e00900017
:104da0001000be00e00f5000e08f580003003a00f2
:104db00050012000000f7800410037001e009000d5
:104dc00020609000e14f500010003a003e0090003b
:104dd0001001be008040eb0084ff20000500200091
:104de0001e009000100907000001be00f0ff2f0018
:104df00001002000800f5100818f590026003a00e9
:104e000090002000000f7800230037001e00900063
:104e100020609000e24f500010003a003e009000e9
:104e20001001be008040eb0084ff2f000500200031
:104e30001e009000fc0807000001be00f0ff2f00dc
:104e400001002000800f5100818f590012003a00ac
:104e500090002000000f78000f0037003e00900007
:104e60001001be008040eb0084ff2f00f5ff200002
:104e70001e009000ec0807000001be00f0ff2f00ac
:104e8000f1ff2000800f5100818f590002003a008d
:104e900090002000000f78001e0078000000e00065
:104ea00007003a003e0090001000be000001be0066
:104eb0001e009000050007000080fb00000f780036
:104ec0001e0078000080fa00000006000e00fa00c4
:104ed0004007980052079800630798000040eb00d5
:104ee000604798005e019000ee0190004e00900037
:104ef0008200070010079800210798001cc8bf0017
:104f00000004e00005003200910207000004e00008
:104f10000200320090c0b300310037001a28ef00c1
:104f20001ec8bf000004e0000b003a004e009000d5
:104f30009080fb00104090000080fb004800dd00e6
:104f400000807000022020008000eb0099ed070037
:104f500010c0b3001ee8b7000040eb00004f78001f
:104f6000170037004e0090009080fb00104090002a
:104f70000080fb004800dd00008070000002780027
:104f80001e009000ae0090001e019000ae01900047
:104f900061014100e0814900120798002307980051
:104fa0008041eb00040178006b210700e14f5000c5
:104fb0000200320090c0b300604798001e4fe80026
:104fc0004e009000106090009e4f5000030036008d
:104fd0006e4090000004e000e2ff32006e4090005e
:104fe0000080fa00000006000400fa00000f7800bc
:104ff000110798001e0090001e004000104078002d
:105000000080fa00000006000800fa00200798005f
:1050100031079800ae0090003e00900000804000f4
:10502000104f78003e0090000000e800ae009000b5
:105030000080400090407800114798001e4090008a
:105040000080fb00100798001e0090004800dd0063
:10505000100798001e80fb009e0090000100700069
:10506000100798001e0090000080fa000000060063
:105070000c00fa004007980051079800de009000ed
:105080004e009000e0ff0700000f78005e009000e7
:105090000080e800800078004e009000daff0700f2
:1050a000100798001e0090008000eb002007980079
:1050b000310798002e009000be009000c000dd0077
:1050c0000000200020079800310798001e0078009b
:1050d0008000eb002e019000be01900000007100e6
:1050e0008180710020079800310798002e00900001
:1050f000be0090000080fa00000006000a00fa00de
:105100002007980032079800430798002e0090006f
:10511000206090000080fb00e30f500022003a0066
:105120003e009000ce00900062015000e0815800e7
:105130002e009000106090000080fb008000eb00cb
:10514000009ab90004027800028bb9008602780048
:10515000050242000010b8000102420084007800fd
:105160002e029000e44a90008582fb00744b900070
:105170000683fb004833dd0086827200050178005b
:10518000845290008582fb00145290000482fb0040
:105190004822dd000482720084017800021f400072
:1051a00003974800420037003e009000ce00900078
:1051b000e00f5000e08f5800070032003e019000e1
:1051c000ce0190001000200001002000800f51004f
:1051d000818f590014003a002e019000a2499000de
:1051e0008381fb00324a90000482fb004822dd00ec
:1051f0008481710003007800c24990008381fb0024
:10520000524990000281fb004811dd0002817100cb
:10521000820078003e019000ce019000021f400005
:1052200003974800220037003e009000ce00900017
:1052300062015000e08158002e0090001060900044
:105240000080fb008000eb00009ab90004027800a7
:10525000028bb90086027800050242000010b800f7
:1052600001024200840078002e029000e44a90007f
:105270008582fb00744b90000683fb004833dd0001
:105280008682720005017800845290008582fb00be
:10529000145290000482fb004822dd000482720058
:1052a00084017800021f40000397480000000000be
:1052b0001e00be000080fa00000006000800fa0090
:1052c00020079800614798002468ef006e40900026
:1052d0008080fb0080fd2f00008060000000e00067
:1052e00004003200f0c1b30024e8b7000080eb00f6
:1052f000390037002e0090004010900010079800f1
:105300002e00900080189000701090002e019000e8
:1053100010199800211998000e80e800800078008c
:105320002e009000d3fa0700000f78001e007800ce
:105330000000e00004003a00b0c1b30024e8b70068
:105340000080eb00240037001e00780030489000f9
:105350000080fb00680060000000e00004003200f4
:10536000f0c1b30024e8b7000080eb001a0037005a
:105370002e00900060109000700060000000e000bf
:10538000060032006e4090000044a0008080fb00c8
:105390002e00900061109800040037006e409000cd
:1053a0008080fb002e009000611098000e80e800c5
:1053b000800078002e009000d4f407000004e00084
:1053c00004003a0090c0b30024e8b7000080eb006e
:1053d000010037000000eb000080fa00000006002a
:1053e0002400fa00600f9800710f980002179800cf
:1053f00013179800fe0890000e1090000088b90066
:10540000000078008000eb00008fbe00ee089000e6
:10541000210798000000eb00300798000000eb0027
:10542000100f98001e10900030089000610060007e
:105430000000e00006003a00d0c1b30024e8b70045
:1054400090002000300798000000eb003e0137007c
:105450001e00be00e00f5000e08f580002003a002e
:105460000000eb0038013700b92007000004e0001d
:105470000600320080c1b30024e8b700800120009c
:10548000300798000000eb002f0137001e68ef0086
:105490001e10900010017800320f98001e1090002e
:1054a000e0019000430798001e10900070019000ea
:1054b0008009900052079800630798001e10900022
:1054c000c0009000300090000001be003e08900037
:1054d0000aff0700400f9800510f98001e1090001f
:1054e000500090008000eb004e099000de09900013
:1054f0000200400083804800400f9800510f980040
:10550000d14080001e109000808f50000c003200af
:105510001cc8bf000004e000070032000c010700b7
:105520000004e0000400320090c0b30024e8b7009b
:105530000000eb00040137009e119000d34088006a
:1055400082418000934180004e089000de08900068
:10555000800f5100818f59001f0032001cc8bf000e
:105560000004e00007003200f90007000004e0003a
:105570000400320090c0b30024e8b7000000eb0044
:10558000f10037001e68ef003e0890009080fb009d
:10559000104090000080fb004800dd00008070009b
:1055a000000178004e089000de089000731f07008d
:1055b0000004e00004003a00b0c1b30024e8b700e2
:1055c00080002000300798004e099000de0990000e
:1055d00082418800934188001e10900010099000bd
:1055e000a009900072079800030f9800bd003700d3
:1055f0005e019000ee0190007e0090008e08900009
:10560000800f5100818f590004003a009e109000d5
:10561000310890000020a000b00898004e009000d3
:105620006102b8003e099000825990008381fb001e
:10563000125b90000683fb004833dd008681710019
:1056400003007800a25990008381fb00325990003a
:105650000281fb004811dd000281710082007800a8
:10566000800f5200818f5a006f003a0010c0b300c3
:10567000405798001cc8bf000004e000070032003b
:10568000b30007000004e0000400320090c0b30043
:1056900024e8b7000000eb00ab0037000000eb008f
:1056a000400798001e109000500090008000e80015
:1056b0001e109000510098001e109000d000900025
:1056c0003e089000106090000080fb00808f50002a
:1056d00016003a001e1090008000eb005100980068
:1056e0001e10900030089000640060000000e00090
:1056f000080032008040eb001e1090006cf707009d
:105700000080fb00300798000040eb0040579800f5
:105710000600370012002000030020001e10900039
:10572000e5ee07000080fb00300798003e00900087
:10573000f50f500004003a0050c1b30024e8b70050
:105740000000eb00800037003e0090000000e00009
:1057500035003a001e109000c0009000300090000c
:105760000001be003e08900064fe0700400f980054
:10577000510f98001e109000500090008000eb0028
:105780004e099000de09900002004000838048002e
:10579000400f9800510f98009e119000d340880050
:1057a0004e5090000004e0001b0032003e089000c4
:1057b0009080fb00104090000080fb004800dd005e
:1057c00000807000000178004e089000de08900014
:1057d000ea1e07000004e0000a003a00b0c1b3006e
:1057e00024e8b70080002000300798000080eb001c
:1057f0008080eb0080418800914188000000eb0030
:10580000510037004e099000de0990008241880067
:1058100093418800040037004e099000de09900093
:1058200082418800934188003e0090000000e00023
:105830002c003a003e0890009080fb001040900041
:105840000080fb004800dd000080700080007800d0
:105850004e00900000804000ae0090009140780023
:10586000014878004e0090000000e80040079800d2
:105870002e0090000000e800200798005e009000d5
:10588000ee00900061004000e08048005007980062
:10589000610798000081eb008081eb001e0f410042
:1058a0005e9749001e0890000000e800100f980065
:1058b0001e10900030089000640060000000e000be
:1058c000060032007e0090008e08900061004000cb
:1058d000e080480070079800010f980010c0b300e6
:1058e0001ce8b7003e0090000000e00004003a0011
:1058f0001e00be00e00f5000e08f58003cff3a0051
:105900001e109000ce019000630098001e109000c1
:105910005e019000ee01900072009800030898006c
:105920001e1090007e0190008e09900012089800d1
:10593000230898009e0890007e089000800178005f
:10594000110009008380d8000080fa0000000600e2
:105950000800fa00d1408000010f78001e00780096
:1059600090007800110798001e007800c000900099
:10597000300090000001be001e009000dffd070017
:1059800020079800310798001e0078005000900012
:105990008000eb002e019000be019000020040004c
:1059a0008380480020079800310798001e0090006f
:1059b0009080fb00104090000080fb004800dd005c
:1059c000008070008041eb00000178002e00900004
:1059d000be009000e01e07000004e00002003a0054
:1059e00090c0b300020037001c68ef000040eb00dd
:1059f0000080fa00000006000200fa00000f7800a4
:105a00002468ef001e00780070019000800990006b
:105a10001e007800a00890001008900000006900a7
:105a2000818069000080700000f0a7000000ea009b
:105a30000000e9004f00de000080fa0000000600d0
:105a40001e00fa00300f9800410f9800520f980086
:105a5000630f9800ce0890005e0890000088b9009f
:105a6000000078008000eb00008fbe00be089000b0
:105a7000210798000000eb00700798000000eb0081
:105a8000600798002468ef006e089000100178000d
:105a9000020f98006e089000e001900053079800f4
:105aa0006e08900070019000800990003207980005
:105ab000430798006e089000300890006200600074
:105ac0000000e00004003a00e0c1b30024e8b700a1
:105ad0000000eb00e40037001cc8bf000004e00039
:105ae000070032009aff07000004e00004003200c3
:105af00090c0b30024e8b7000000eb00da003700e4
:105b0000d14080006e089000808f5000c5003200a8
:105b10005e0090006102b8000e099000825990006a
:105b20008381fb00125b90000683fb004833dd009d
:105b30008681710003007800a25990008381fb00e8
:105b4000325990000281fb004811dd000281710092
:105b500082007800800f5200818f5a00b10032001d
:105b6000ee099000d34088006e089000c0009000bd
:105b7000300090000001be000e0890005ffd07009d
:105b8000100f9800210f98006e08900050009000b0
:105b90008000eb001e099000ae099000020040005a
:105ba00083804800100f9800210f98001e68ef00b6
:105bb0000e0890009080fb00104090000080fb00d9
:105bc0004800dd0000807000000178001e08900091
:105bd000ae089000e91d07000004e00006003a004e
:105be00080c0b30024e8b700800020007007980050
:105bf0000000eb009c0037001e099000ae099000e9
:105c00008241880093418800860037006e0890002a
:105c100010099000a00990003e009000ce00900076
:105c2000800f5100818f590005003a00d0c3b300a6
:105c300024e8b700d0032000700798007d003700eb
:105c40005e0090006102b8000e0990008259900039
:105c50008381fb00125b90000683fb004833dd006c
:105c60008681710003007800a25990008381fb00b7
:105c7000325990000281fb004811dd000281710061
:105c800082007800800f5200818f5a0046003a004f
:105c90000000eb00500798006e0890005000900044
:105ca0008000e8006e089000510098006e08900097
:105cb000d00090000e089000106090000080fb0063
:105cc000808f50000f003a006e0890008000eb00bb
:105cd0005100980012002000030020006e08900080
:105ce00075ed07000080fb00700798007e009000b3
:105cf0000000e00003003200f0c0b30024e8b70069
:105d00004c0037006e089000c000900030009000fa
:105d10000001be000e089000f8fc0700100f98006c
:105d2000210f98006e089000500090008000eb005a
:105d30001e099000ae0990000200400083804800d8
:105d4000100f9800210f9800ee099000d3408800b2
:105d50001e68ef000e0890009080fb00104090003d
:105d60000080fb004800dd0000807000000178002a
:105d70001e089000ae089000801d07000004e0009f
:105d800005003a0080c0b30024e8b700800020007e
:105d900070079800270037001e099000ae09900098
:105da00082418800934188000e0890009080fb009b
:105db000104090000080fb004800dd000080700073
:105dc000800078005e0090000080400090407800e5
:105dd0002e009000014878005e0090000000e8006e
:105de000500798002e0090000000e800200798005f
:105df0003e009000ce00900061004000e08048002e
:105e000030079800410798006e0090000000e800fd
:105e1000600798000081eb008081eb001e0f4100bd
:105e20005e9749001e00be00e00f5000e08f580052
:105e300076ff3a006e089000de0190006300980043
:105e40006e0890003e019000ce0190007200980014
:105e500003089800ee0090004e0890008001780042
:105e6000110009008380d8000080fa0000000600bd
:105e70001c00fa00881f7800300f9800410f98002e
:105e8000225f98000040eb0020479800090037008f
:105e90002e4090000080fb00ce0890000080400063
:105ea00001c2b300014878002e4090000040e80095
:105eb000204798002e409000ea4f5000f4ff360033
:105ec0003e08900090407800e0c2b30080cf5000c0
:105ed000040032003e089000104078000004e0000a
:105ee00002003a000040eb005e0037003e089000e0
:105ef000c7e90700200798002e009000ec0f500023
:105f000009003e0066004700be089000bae907009d
:105f100066004700ae589000c60007000004e0008d
:105f200003003200040037000040eb004d00370052
:105f30000040eb004b00370066004700e102200004
:105f4000a3e90700000f78001e0078000000e000c1
:105f50000a0032001e0078008040eb000148780003
:105f60001e0fe8001e007800a9e90700e30f5000ab
:105f7000020036000040eb003a00370066004700a0
:105f8000a3e90700e80f5000020036000040eb00d4
:105f9000340037000040eb00204798000d00370028
:105fa0002e4090000080fb00ce0890000080400052
:105fb000ae4090008180fb006601470081004100f7
:105fc00091407800014878002e4090000040e800a1
:105fd000204798002e4090000084fb006600470098
:105fe0008be90700800f5400edff39001e00780098
:105ff0000000e0001a0032001e0078001040780017
:106000000004e000160032000040eb00204798003a
:106010000d0037002e4090000080fb00680040001b
:10602000ce08900000804000ae4090008180fb00d0
:106030009e80400091407800014878002e409000fa
:106040000040e800204798002e4090000084fb00ac
:106050001e0078006ee90700800f5400edff390044
:1060600010c0b3004f0478000080fa000000060062
:106070001200fa0070079800015798008e509000a7
:106080007e0090006b0007000004e00002003a0070
:106090000040eb00650037000040eb00004f780047
:1060a000080037001e80fb009e80fb007e019000f0
:1060b0008100410091407800000047002140980095
:1060c0001e4fe8001e407800e74f50000d003e00d4
:1060d0001e80fb00fe009000008040009040780091
:1060e000e0c2b30080cf5000060032001e80fb00eb
:1060f000fe00900000804000104078000004e000a6
:10610000e8ff3a009e4078001147980005003700ec
:106110001e80fb000000470001c2b3002140980030
:106120001e4fe8001e407800e74f5000f8ff360091
:106130001e4090000080fb00fe00900000804000a8
:1061400090407800e0c2b30080cf50001d003a00bc
:106150001e4090000040e800104798000c003700f7
:106160001e80fb009e4090008180fb007e0190001d
:1061700081004100914078000000470021409800d4
:106180001e4fe8001e4090000040e80010479800b5
:106190001e4090000080fb00fe0090000080400048
:1061a000104078000004e000edff3a0005003700e1
:1061b0001e80fb000000470001c2b3002140980090
:1061c0001e4fe8001e407800ea4f5000f8ff3600ee
:1061d0000040eb00504f9800ae40900000c2b3006a
:1061e00080cf500002003a00f0c5b300204798006d
:1061f0000040eb00004f7800080037001e80fb00d5
:10620000fe009000008040009e80fb00810047005f
:10621000a1409000014878001e4fe8001e40780021
:10622000eb4f5000f5ff360010c0b3000080fa00bd
:10623000000006000a00fa0030079800014f98009d
:106240000040eb00204798003e009000f0e8070077
:10625000200798000000eb00000f7800aa0037002c
:106260001e007800be009000008040009040780042
:1062700000c2b30080cf500006003c001e00780032
:10628000be0090000080400010407800e54f5000b4
:1062900065003a001e007800be00900000804000bb
:1062a0009040780020c2b30080cf50005e003200e2
:1062b0001e007800be0090000080400090407800f2
:1062c000b0c2b30080cf5000570032001e007800eb
:1062d000be0090000080400090407800c0c2b30033
:1062e00080cf5000500032001e007800be009000a9
:1062f0000080400090407800f0c2b30080cf500092
:10630000490032001e007800be009000008040006e
:1063100090407800a0c3b30080cf5000420032000c
:106320001e007800be009000008040009040780081
:10633000b0c3b30080cf50003b0032001e00780095
:10634000be0090000080400090407800c0c3b300c1
:1063500080cf5000340032001e007800be00900054
:106360000080400090407800d0c3b30080cf500040
:106370002d0032001e007800be009000008040001a
:1063800090407800e0c3b30080cf50002600320078
:106390001e007800be009000008040009040780011
:1063a000b0c5b30080cf50001f0032001e0078003f
:1063b000be0090000080400090407800c0c5b3004f
:1063c00080cf5000180032001e007800be00900000
:1063d0000080400090407800d0c5b30080cf5000ce
:1063e000110032001e007800be00900000804000c6
:1063f00090407800c0c7b30080cf50000a00320040
:106400001e007800be0090000080400090407800a0
:10641000e0c2b30080cf500005003a002e4090004b
:10642000e14f500002003a000040eb003b00370013
:106430000e4890000004e00010003a001e007800b2
:10644000be0090000080400090407800a0c2b300e1
:1064500080cf5000070032001e007800be00900080
:106460000080400090407800f0c3b30080cf50001f
:1064700002003a000040eb00280037001e007800c0
:10648000be0090000080400090407800e0c2b30061
:1064900080cf500002003a0010c0b300204798009f
:1064a0001e007800be009000008040009040780000
:1064b00000c6b30080cf5000120034001e007800e8
:1064c000be0090000080400090407800a0c7b3005c
:1064d00080cf50000b003c001e007800be009000f2
:1064e000008040009e0078003e0190008100410045
:1064f000914078000141780001ceb3008140410015
:10650000014878001e0fe8002e0090009e007800e1
:10651000808f500052ff350010c0b3000080fa0099
:10652000000006001800fa00000f9800120f9800f3
:10653000230f9800310f98001e099000ae099000bb
:10654000028fbe000e08900090017800230798008b
:106550003e089000e10f500003003200e20f5000af
:1065600009003200100037000e0890007001900002
:10657000800990001e00be00020040008380480099
:10658000008fbe00080037000e0890001009900030
:10659000a00990001e00be0000005100818059003b
:1065a000008fbe00000000001cc8bf000004e00017
:1065b00007003200e6fc07000004e000040032009f
:1065c00090c0b30024e8b7000080eb000d01370055
:1065d0000e08900010019000a00190003207980072
:1065e000430798000e0890003e019000ce019000f5
:1065f00032009800430098000e08900010099000a7
:10660000a009900032079800430798001e01be00c1
:106610003e009000ce009000800f5100818f590005
:1066200004003600f0c1b30024e8b7000080eb009e
:10663000f40037008e089000310890000020a1007f
:10664000b00898001e00be000e099000700198006e
:10665000010998001e02be002e0190008259900090
:106660008381fb00125b90000683fb004833dd0052
:106670008681710003007800a25990008381fb009d
:10668000325990000281fb004811dd000281710047
:10669000820078000001be000400be00b5e70700dc
:1066a00050079800610798001e02be002e0190005e
:1066b000825990008381fb00125b90000683fb00ef
:1066c0004833dd008681710003007800a2599000f4
:1066d0008381fb00325990000281fb004811dd00ec
:1066e00002817100820078005e0190000191b90082
:1066f00002017800ee019000009bb900860178004d
:1067000003014100de0190000018b80001014100c2
:10671000820078000000520081805a00008fbe0085
:106720009e0078000e089000610098002e009000f6
:10673000106090000080fb008000eb000001be00b4
:106740005e009000ee0090008ae707003007980096
:10675000410798002e009000106090000080fb0020
:106760008000eb003e0190000191b9000201780029
:10677000ce019000009ab900840178000301410025
:10678000be0190000018b8000101410082007800ad
:106790005e019000ee0190000000510081805900e0
:1067a0005007980061079800de0090000e089000e6
:1067b000510098003e009000ce009000e00f500085
:1067c000e08f5800620032003e019000ce01900040
:1067d0000e089000b8ea0700604f98006e489000dd
:1067e0000004e0005a003200ee489000c0c3b3003d
:1067f00080cf500052003a000e0890003008900000
:10680000610060000000e0001e0032000e089000f1
:10681000a0009000100090000e0990003001980038
:10682000410198003e019000ce0190001000200030
:1068300001002000800f5100818f590008003200b4
:106840003e009000ce00900061005000e0805800b3
:106850000001be000e08900097ea0700604f980004
:106860008040eb000e08900011f307000004e000e8
:1068700037003200f0c0b30024e8b7000080eb001e
:10688000600037000e089000a000900010009000fb
:106890000e09900030019800410198003e009000e0
:1068a000ce00900061005000e08058000001be0062
:1068b0000e08900080ea0700604f98006e48900034
:1068c0000004e00004003200f0c0b30024e8b70088
:1068d0000080eb004b0037002e01900082599000a1
:1068e0008381fb00125a90000482fb004822dd00e5
:1068f0008481710003007800a25990008381fb001d
:10690000325990000281fb004811dd0002817100c4
:1069100082007800800078000e08900061009800e6
:106920002e009000106090000080fb000000e90045
:10693000800078000e089000510098000400370095
:10694000f0c0b30024e8b7000080eb002d00370052
:106950000e089000c0009000300090000001be00c2
:106960002e009000e5f907003007980041079800d5
:106970000e089000500090008000eb005007980037
:10698000610798003e019000ce0190005e009000eb
:10699000ee0090000200400083804800300798001d
:1069a000410798001a28ef001e68ef002e009000a3
:1069b0009080fb00104090000080fb004800dd004c
:1069c00000807000000178003e009000ce00900032
:1069d0006a1a07000004e00004003a00b0c1b300e6
:1069e00024e8b7000080eb00060037003e0190006d
:1069f000ce01900082418800934188002468ef0016
:106a00000000eb000080fa00000006002000fa0001
:106a1000889fbe00500f9800620f9800730f980077
:106a20006000b80030079800410798001e68ef002a
:106a30005e089000206090000080fb00e10f500095
:106a400015003200e30f500035003a006e09900047
:106a5000fe0990004218dd00ce10de0081007000bb
:106a60004210dd0010079800210798000040eb005d
:106a7000004f7800f0ff2f00f1ff20005007980032
:106a80006107980080ff2f00f1ff20007007980039
:106a9000010f9800330037007e0890006300b900b2
:106aa000000178006e0890006000b90000007800d6
:106ab00000014100ee089000300020000008b800fe
:106ac000010141008200780010079800210798001a
:106ad00010079800210798001e00900000407800e1
:106ae000614f60001e009000ae0090008100d10058
:106af0000080d3001007980021079800f0ff2f00b6
:106b000001002000500798006107980080ff2000d6
:106b10000100200070079800010f98001100370055
:106b20006e089000fe089000000040008180480040
:106b300010079800210798000040eb00004f7800f4
:106b4000f0ff2f0001002000500798006107980017
:106b500080ff2f000100200070079800010f9800af
:106b6000000000005e089000e04090008180fb0083
:106b7000704190000281fb004811dd0082807000ae
:106b800001047800804890008180fb00104890004c
:106b90000080fb004800dd00008070008004780069
:106ba0005e099000825990008381fb00125a900088
:106bb0000482fb004822dd0084817100030078001c
:106bc000a25990008381fb00325990000281fb00a2
:106bd0004811dd0002817100820078000001be00d2
:106be0001e009000ae00900062e607000800400022
:106bf00089804800100f9800210f98005e099000ce
:106c0000825990008381fb00125a90000482fb009d
:106c10004822dd008481710003007800a2599000b1
:106c20008381fb00325990000281fb004811dd0096
:106c3000028171008200780061005000e0805800fd
:106c40001e019000ae01900002027800030178005e
:106c500080017800010078000302620000006100fa
:106c60008000eb00c000dd00000020000001be003d
:106c70006120b80000017100818171001207980045
:106c80002307980062418000734180001e08900035
:106c9000ae089000800f5100818f5900ae003a007d
:106ca0005e08900020609000e34f500007003a001b
:106cb00001a420001e009000008040001001be00d2
:106cc0003207980043079800470137005e0890009c
:106cd00020609000e24f500008003a0001a420001c
:106ce0001e00900000804000100078008000eb0043
:106cf00030079800410798003b0137005e0890007c
:106d000020609000e14f500037013a009e00900053
:106d100000a4200000804000104078000080fb00ac
:106d20008000eb0030079800410798001e40780073
:106d30000004e000080032003e009000ce00900009
:106d4000cc09dd004400de0000807100c408de00d4
:106d500030079800410798001e009000ae00900098
:106d600061024000e08248005e0990008259900074
:106d70008381fb00125b90000683fb004833dd003b
:106d80008681710003007800a25990008381fb0086
:106d9000325990000281fb004811dd000281710030
:106da0008200780061005000e08058000403780001
:106db000050178008001780001007800030263007b
:106dc000000061008000eb00c000dd00000020003a
:106dd0000001be006120b8000001710081817100d6
:106de00012079800230798001e009000ae00900044
:106df000e00f5000e08f580023003a0018c8bf0091
:106e00000004e0000b00320011c0b3006022b800a3
:106e10006011b8005e08900003010700e00f500009
:106e2000e08f5800030032005e009000ee009000fa
:106e3000fa0037001e089000ae0890006100400084
:106e4000e080480002a420004c1907000004e00084
:106e500007003a00f0ff2f00010020006041880089
:106e6000714188005e009000ee009000eb0037005a
:106e70001e089000ae08900061004000e0804800cd
:106e800060418800714188009e00900000a42000ad
:106e900000804000104078000080fb008000eb0084
:106ea000300f9800410f98001e4078000004e00069
:106eb0000d0032003e099000ce0990004418dd001c
:106ec000cc10de00810070004410dd003e01900017
:106ed000ce019000020040008380480030079800f7
:106ee00041079800c00037003e099000ce0990008d
:106ef000f000200001002000020278000301780069
:106f00008001780001007800030262000000610047
:106f10008000eb00c000dd00000020000001be008a
:106f20006120b80000017100818171004818dd0006
:106f3000c810de00810070004810dd003e019000a6
:106f4000ce01900002004000838048003007980086
:106f500041079800a400370018c8bf000004e000f3
:106f60000b00320011c0b3006022b8006011b800fd
:106f70005e089000ac000700e00f5000e08f580062
:106f8000030032005e009000ee009000a300370086
:106f900002a420001e089000ae089000f718070019
:106fa0000004e00007003a00f0ff2f00010020007d
:106fb00060418800714188005e009000ee00900002
:106fc000960037001e099000ae09900062418800cb
:106fd000734188005e08900020609000e34f5000ed
:106fe00007003a0001a420001e009000008040002d
:106ff0001001be0032079800430798007a0037005e
:107000005e08900020609000e24f500008003a00b7
:1070100001a420001e0090000080400010007800b5
:107020008000eb0030079800410798006e003700a1
:107030005e08900020609000e14f50006a003a0026
:107040009e00900000a420000080400010407800c6
:107050000080fb008000eb0030079800410798009b
:107060001e4078000004e000080032003e0090005e
:10707000ce009000cc09dd004400de0000807100ed
:10708000c408de0030079800410798001e009000f9
:10709000ae00900061024000e08248005e0990006e
:1070a000825990008381fb00125b90000683fb00f5
:1070b0004833dd008681710003007800a2599000fa
:1070c0008381fb00325990000281fb004811dd00f2
:1070d000028171008200780061005000e080580059
:1070e0000403780005017800800178000100780031
:1070f00003026300000061008000eb00c000dd00bf
:10710000000020000001be006120b80000017100f5
:107110008181710012079800230798009e0090005b
:1071200000a4200000804000104078000080fb0098
:107130008000eb00300f9800410f98001e4078004f
:107140000004e0000d0032003e099000ce099000de
:107150004418dd00cc10de00810070004410dd001a
:107160003e019000ce019000020040008380480064
:1071700030079800410798001b0037003e09900037
:10718000ce099000f00020000100200002027800eb
:10719000030178008001780001007800030262009a
:1071a000000061008000eb00c000dd000000200056
:1071b0000001be006120b8000001710081817100f2
:1071c0004818dd00c810de00810070004810dd00a6
:1071d0003e019000ce0190000200400083804800f4
:1071e00030079800410798003e019000ce019000c2
:1071f0007e0090008e089000800f5100818f590012
:10720000040039007e0190008e099000320798003a
:10721000430798003e009000ce0090004f04be004f
:107220000080fa00000006002000fa00889fbe00df
:10723000200f9800320f9800430f9800540f9800c9
:10724000650f9800615f98002e0890002060900004
:10725000e34f50000b0032002e0890002060900099
:10726000e24f5000070032002e089000206090008e
:10727000e14f500003003200f0ff2f00f1ff20002b
:107280000e0237002e089000206090000080fb0066
:10729000e30f500005003a00f0ff2f00f1ff20003f
:1072a000600798007107980005003700f0ff2f0075
:1072b000010020006007980071079800000000009e
:1072c0001e68ef006e5890000004e0002e003200af
:1072d0000040eb00004f7800624180007341800065
:1072e0004207980053079800200037008041eb00c8
:1072f00002a420004e009000de00900096180700c7
:107300000004e00003003a006e009000fe009000d0
:10731000ea0137001e4fe8002e099000c259900084
:107320008381fb00525a90000482fb004822dd005a
:107330008481710003007800e25990008381fb0092
:10734000725990000281fb004811dd00028171003a
:10735000820078004e019000de01900002004000a3
:107360008380480040079800510798002e0890003d
:10737000006090009e4f5000dcff3e001868ef0058
:107380006000b800cd0137002e089000206090000a
:107390000080fb00e10f50000d003200e30f5000b1
:1073a00026003a003e099000ce0990004218dd0008
:1073b000ce10de00810070004210dd002007980032
:1073c000310798000040eb00104798002400370078
:1073d0004e0890006300b900000178003e0890005c
:1073e0006000b9000000780000014100be08900074
:1073f000300020000008b800010141008200780040
:10740000200798003107980020079800310798005e
:107410002e00900000407800614060001047980006
:107420002e009000be0090008100d1000080d300ab
:107430002007980031079800090037003e089000a7
:10744000ce0890000000400081804800200798008e
:10745000310798000040eb00104798000000000042
:107460002e089000e04090008180fb007041900069
:107470000281fb004811dd00828070000104780069
:10748000804890008180fb00104890000080fb0045
:107490004800dd0000807000800478002e09900014
:1074a000825990008381fb00125a90000482fb00f5
:1074b0004822dd008481710003007800a259900009
:1074c0008381fb00325990000281fb004811dd00ee
:1074d00002817100820078000001be002e00900041
:1074e000be00900023e407000800400089804800a7
:1074f000000f9800110f98002e09900082599000fb
:107500008381fb00125a90000482fb004822dd00b8
:107510008481710003007800a25990008381fb00f0
:10752000325990000281fb004811dd000281710098
:107530008200780061005000e08058002e01900029
:10754000be019000020278000301780080017800fb
:107550000100780003026200000061008000eb007f
:10756000c000dd00000020000001be006120b80066
:107570000001710081817100220798003307980093
:1075800062418000734180000e0890009e089000c8
:10759000800f5100818f59004000320018c8bf0091
:1075a0000004e0002c0032000040eb00004f7800a7
:1075b00062418000734180004207980053079800a1
:1075c000200037008041eb0002a420004e00900014
:1075d000de009000e01707000004e00003003a001e
:1075e0006e009000fe009000340137001e4fe8004e
:1075f0002e099000c25990008381fb00525a9000de
:107600000482fb004822dd008481710003007800c1
:10761000e25990008381fb00725990000281fb00c7
:107620004811dd0002817100820078004e01900057
:10763000de0190000200400083804800400798006f
:10764000510798002e089000006090009e4f500057
:10765000dcff3e001868ef0002a420000e08900036
:107660009e089000451707000004e00007003a005c
:10767000f0ff2f0001002000604188007141880068
:107680006e009000fe0090000c0137000e09900083
:107690009e09900062418800734188002e08900086
:1076a00020609000e34f500054003a00ae0090007c
:1076b00000a4200000804000de0890008140780097
:1076c000014878002e0090008000e80000a420000f
:1076d000008240005e099000ee09900000f02f004b
:1076e0000100200082027800030178008001780008
:1076f0000100780083826200000061008000eb00de
:10770000c000dd00000020000001be006128b800bc
:107710000001710081817100c81add004810de008f
:1077200000807200c818de0000407800004a78002f
:107730002e0090008080e80000a42000008240001d
:107740005e099000ee09900000002000f10f20007b
:10775000820278000301780080017800010078003f
:1077600083826200000061008000eb00c000dd0049
:10777000000020000001be006128b8000001710077
:10778000818171004018de00010020000040780077
:10779000004a78002e009000e300400000a4200082
:1077a000008240005e099000ee0990000000200079
:1077b00001f0200082027800030178008001780047
:1077c0000100780083826200000061008000eb000d
:1077d000c000dd00000020000001be006128b800ec
:1077e00000017100818171004818de000100200055
:1077f00000407800004a7800ad0037002e08900065
:1078000020609000e24f500022003a00ae0090004d
:1078100000a4200000804000de0890008140780035
:10782000014878002e0090008000e80000a42000ad
:10783000008240005e099000ee09900000f02f00e9
:1078400001002000820278000301780080017800a6
:107850000100780083826200000061008000eb007c
:10786000c000dd00000020000001be006128b8005b
:107870000001710081817100c81add004810de002e
:1078800000807200c818de0000407800004a7800ce
:10789000870037002e08900020609000e14f5000d4
:1078a00083003a00ae00900000a420000080400059
:1078b00090407800214798001e4090000004e000ae
:1078c000090032005e0890008040780040002000ef
:1078d0008008dd002e4090006f40600000c0700006
:1078e00020479800020037005e089000204798006b
:1078f000ae00900000a42000008040002e419000c7
:10790000024878002e009000be0090006102400006
:10791000e08248002e099000825990008381fb008c
:10792000125b90000683fb004833dd008681710006
:1079300003007800a25990008381fb003259900027
:107940000281fb004811dd00028171008200780095
:1079500061005000e08058000403780005017800c1
:1079600080017800010078000302630000006100dc
:107970008000eb00c000dd00000020000001be0020
:107980006120b80000017100818171002207980018
:10799000330798002e009000be009000e00f5000ca
:1079a000e08f580020003a0011c0b3006022b800f8
:1079b0006011b8002e0890001bfe0700e00f500079
:1079c000e08f5800030032006e009000fe0090002f
:1079d0003a0037000e0890009e08900061004000b9
:1079e000e080480002a42000641607000004e000c4
:1079f00007003a00f0ff2f000100200060418800de
:107a0000714188006e009000fe0090002b0037004e
:107a10000e0890009e08900061004000e080480041
:107a20006041880071418800ae00900000a42000f1
:107a30000080400090417800234798001e4090004d
:107a40000004e000080032005e089000ee0890009c
:107a5000cc0add004400de0000807200c408de00b5
:107a6000204798000d0037005e089000ee08900057
:107a70004809dd004800de0000007100c808de0093
:107a800000407800ef4060002e41900000cfb3002e
:107a90000040610000c0700020479800ae009000d8
:107aa00000a4200000804000ae4190000348780010
:107ab00010c0b30018e8b7006000b8004f04be0063
:107ac0000080fa00000006000200fa00000f7800b3
:107ad0000001eb009e0078000040eb000200070070
:107ae0000080fa00000006005200fa0040cf980023
:107af00071279800022f980010002000400798007e
:107b0000fe209000110798006a00470020079800a7
:107b1000a0418000800078002e00900078f40700db
:107b20002468ef001e00900010407800004f78009d
:107b30001e4078000004e00004003a00f0c1b300e9
:107b400024e8b7000080eb00ae0137001e80fb0088
:107b5000e1022000810f500004003200c105200026
:107b6000810f5000b8003200030137001e00900062
:107b70000000e800100798001e00900010407800f8
:107b8000004f7800e0c2b3009e40780080cf5000e4
:107b900089003a001e0090000000e80010079800dd
:107ba0001e00900010407800004f78002e009000da
:107bb00070119000801990000041800011418000f8
:107bc000800f5100818f590004003a00f0c1b300ca
:107bd00024e8b7000080eb008a0137002e009000f7
:107be00080189000701090002e01900010199800dd
:107bf00021199800100020004007980068004700f5
:107c000012c0b300800078002e009000a8eb07009f
:107c1000300798003e0090000000e00004003a00a9
:107c2000b0c1b30024e8b7000080eb007501370055
:107c30003e009000a1ea07002e019000701198000c
:107c4000011998002e00900080189000701090008c
:107c50002e01900010199800211998002e00900014
:107c60008018900070109000e00f5000e08f5800d6
:107c70001d003a002e009000c1c5b3004158980085
:107c800010c0b30010479800090037001e40900054
:107c90000080fb00ae0090000080400001c2b300f5
:107ca000415898001e4090000040e800104798009e
:107cb0001e409000ea4f5000f4ff36000041800063
:107cc000114180002e019000101998002119980090
:107cd00000418000114180002e0190007011980039
:107ce00001199800150037002e009000e1c2b30082
:107cf000415898002e009000e1c2b30051589800fe
:107d000020c0b30010479800090037001e409000c3
:107d10000080fb00ae0090000080400001c2b30074
:107d2000415898001e4090000040e800104798001d
:107d30001e409000ea4f5000f4ff36000000eb00b8
:107d4000400798006800470012c0b3008000780028
:107d50002e00900056eb07000000e0000a003a00f9
:107d6000b0c1b30024e8b7000080eb002501370064
:107d70001e0090000000e800100798001e00900010
:107d800010407800004f7800c0c5b3009e407800d6
:107d900080cf5000f6ff32001e4078000004e00063
:107da00028003a00a0418000ae009000d4f3070004
:107db0000000eb00130137001e4078000004e000d3
:107dc00005003a00a0418000ae009000ccf307000f
:107dd0000000eb000b013700c0c5b3009e407800e7
:107de00080cf500013003a00060037001e009000bc
:107df0000000e800100798001e0090001040780076
:107e0000004f7800c0c5b3009e40780080cf50007e
:107e1000f6ff32001e4078000004e00009003a003e
:107e2000a0418000ae009000b5f307000000eb0019
:107e3000f4003700f0c1b30024e8b7000080eb0085
:107e4000f0003700ee0037001e0090000000e80050
:107e5000100798001e00900010407800004f780036
:107e6000c0c5b3009e40780080cf500004003a00a7
:107e7000f0c1b30024e8b7000080eb00e100370058
:107e80001e4078000004e0001e003a00a24180007d
:107e90000041800011418000701198000119980084
:107ea000a24180000041800011418000101998001b
:107eb00021199800a0418000c1c5b3004158980025
:107ec00010c0b3001047980009003700a14180009e
:107ed0001e4090000080fb000080400001c2b30003
:107ee000415898001e4090000040e800104798005c
:107ef0001e409000ea4f5000f4ff36000000eb00f7
:107f0000c000370000418000114180002e01900028
:107f10007011980001199800004180001141800003
:107f20002e01900010199800211998002e00900041
:107f3000c1c5b3004158980010c0b3001047980065
:107f4000090037001e4090000080fb00ae0090004a
:107f50000080400001c2b300415898001e409000cc
:107f60000040e800104798001e409000ea4f500083
:107f7000f4ff3600a20037000040eb0010479800e5
:107f80000e0037001e4090000080fb001e4178006c
:107f9000c1da2000827078001e4090000040e800a6
:107fa000104798001e0090000000e800100798009d
:107fb0001e00900010407800004f78001e407800ae
:107fc0000004e00007003200c0c5b3009e40780006
:107fd00080cf5000030032001e409000eb4f500055
:107fe000e8ff36001e409000ec4f50000e003a00b3
:107ff000060037001e0090000000e80010079800ff
:108000001e00900010407800004f78001e4078005d
:108010000004e00004003200c0c5b3009e407800b8
:1080200080cf5000f3ff3a001e4090000080fb001c
:10803000c1da20000041eb00827078008040eb0044
:10804000c0da20000af807000004e00002003a004d
:108050000080eb006b0037000040eb0010479800f9
:10806000150037001e4090000080fb009e409000ed
:108070008180fb002e019000fc804000e2c078006f
:108080000000470001c098001e4090000080fb00e7
:108090009e4090008180fb00c2da2000e2c07800a0
:1080a0002e01900000004100415898001e409000b1
:1080b0000040e800104798001e409000ea4f500032
:1080c000e8ff3600ae009000c0d120000cf307009e
:1080d0008041eb0012c0b300ae009000c0d1200080
:1080e000e0e207000000e00004003200c0c0b3007e
:1080f00024e8b7000080eb0042003700406a8000af
:10810000f00f500004003200f0c1b30024e8b700c3
:108110000080eb003b0037000040eb001047980068
:108120000e0037001e4090000080fb009e40900033
:108130008180fb007c814000c1d120008100410092
:10814000914078002e0190000000410041589800b5
:108150001e4090000040e800104798001e4090002c
:10816000ea4f5000efff3600f068800001698000a0
:108170002e01900070119800011998002e009000b7
:1081800080189000701090002e0190001019980037
:10819000211998001e4078000004e00013003a0006
:1081a000a0418000ae009000d5f207000000eb0077
:1081b000140037001e0090000000e800100798002f
:1081c0001e00900010407800004f78001e4078009c
:1081d0000004e00005003a00a0418000ae009000dd
:1081e000c7f207000000eb0006003700c0c5b3006f
:1081f0009e40780080cf5000eeff3200000000006b
:1082000052fe37000080fa00000006001e00fa004f
:10821000500f9800610f98005e0890000000e00089
:10822000030032006e089000004078000100370023
:10823000a0c0b300204f9800c0d120006007980074
:108240000040eb00204798000000eb00300798004a
:108250002468ef005e0890000000e00003003a0090
:1082600090db2000000f780009003700de08900046
:10827000010f78006e0890000000e00004003a0052
:10828000f0c1b30024e8b7000000eb00b4013700f0
:108290002e4890000000fb000000e9001e00400096
:1082a00070079800a0418000800078006e00900068
:1082b00093f207006e009000c0589000e0c2b30037
:1082c00080cf5000a0003a006e009000d05890007f
:1082d000e0c2b30080cf50009b003a006e009000d7
:1082e0007011900080199000020f9800130f9800f1
:1082f00010002000400f98006e0090008018900041
:10830000701090006e0190001019980021199800cb
:108310007800470012c0b300800078006e00900023
:10832000e3e90700400798004e0090000000e000dd
:1083300004003a00b0c1b30024e8b7000000eb002d
:10834000870137004e009000dce8070030418800cc
:10835000414188003041800041418000e00f5000e1
:10836000e08f580006003a00004180001141800073
:108370006e019000701198000119980005003700f7
:1083800030418000414180006e01900070119800e2
:10839000011998006e0090008018900070109000f5
:1083a0006e01900010199800211998000000eb0050
:1083b000400f98007800470012c0b300800078009a
:1083c0006e009000bae90700400798004e00900048
:1083d0000000e00004003a00b0c1b30024e8b70098
:1083e0000000eb005e0137004e009000b3e807008c
:1083f0003041880041418800140037004e08900049
:108400000000e800400f9800780047000041eb00b2
:10841000800078006e009000a5e9070040079800f2
:108420004e0090000000e00004003a00b0c1b3002c
:1084300024e8b7000000eb00490137004e0090002f
:108440009ee80700304188004141880032418000a9
:10845000434180000e0890009e089000800f51005c
:10846000818f5900e5ff3a0032418000434180008e
:108470000e0890009e089000800f5100818f5900d7
:108480000c003a004e00900010407800fb4f400076
:10849000daff32004e00900030489000e84f500064
:1084a000d6ff32004e00900030489000ef4f500051
:1084b000d2ff32000000eb002007980015003700c3
:1084c000ce0090002e009000008040009040780088
:1084d0006e0190002e009000000041007c004000e2
:1084e00001487800a2418000ce0090002e0090004c
:1084f00000804000904078002e0090000000410075
:108500007c004000014878002e0090000000e80048
:10851000200798002e009000ea0f5000e8ff34007a
:108520006e0090000e0990009e0990007210980055
:10853000031898006e0090000e0990009e099000ac
:1085400012189800231898006e009000c0589000f0
:10855000c0c5b30080cf50008d003a001e007800e7
:10856000c1c5b300014878001e00e8008040eb0060
:10857000014878001e007800f9003700a0c0b30061
:1085800030479800030037003e4090000040e9006b
:10859000304798003e4090000000fb00ee00900045
:1085a0007c004000e140780000c2b30080cf500062
:1085b000f5ff32003e409000e74f5000300034009d
:1085c000170037003e0090001e004000be409000a3
:1085d0008100fb006e019000fc804000e2c078004a
:1085e000014878003e0090000000e8003007980045
:1085f0003e4090000040e900304798002e4890002f
:108600008000fb003e009000808f500004003a0084
:108610000000eb003007980010c0b300204798001e
:108620003e409000e74f5000e6ff3c003e009000c7
:108630001e004000e1c2b300014878003e009000f7
:108640000000e800300798002e4890008000fb00f2
:108650003e009000808f50000b003a000000eb00bd
:108660003007980010c0b30020479800070037007b
:108670003e4090000040e90030479800030037007a
:108680000000000001003700000000003e409000a4
:108690000000fb00ee0090007c004000e14078000c
:1086a00000c2b30080cf5000f1ff32001700370046
:1086b0003e0090001e004000be4090008100fb0084
:1086c0006e019000fc804000e2c078000148780014
:1086d0003e0090000000e800300798003e40900007
:1086e0000040e900304798002e4890008000fb00d1
:1086f0003e009000808f500004003a000000eb0024
:108700003007980010c0b300204798003e4090000a
:108710000004e000e6ff3d003e0090001e00400027
:10872000c1c5b300014878003e0090000000e80099
:10873000300798002e4890008000fb003e0090001b
:10874000808f500004003a000000eb0030079800d2
:1087500010c0b300204798006e0090008018900071
:10876000701090006e019000101998002119980067
:108770006e0090007c0007000004e000050032005d
:1087800080c0b30024e8b7000000eb00740037009d
:10879000000000006e0090007011900080199000a1
:1087a0000041800011418000800f5100818f5900ed
:1087b00072ff3a003e0090000000e9003007980088
:1087c0000000eb00200798002e4090000004e0001d
:1087d00041003200be019000230f980014003700c2
:1087e0002e0090001e0040009040780061579800d5
:1087f0002e0090001e004000be0090009e804000b1
:1088000091407800014878003e0090001e00400032
:108810006e519000024878003e0090000000e90090
:10882000300798002e0090000000e8002007980014
:10883000be0090002e009000008050000000e0007c
:10884000e7ff3c002e0890000000e8002007980099
:10885000fe0090001e007800008050003007980055
:10886000140037002e0090001e0040009041780058
:10887000635798002e0090001e004000be0090003c
:108880009e80400091407800014878003e009000b2
:108890001e004000ee509000014878003e0090001d
:1088a0000000e900300798002e0090000000e8006a
:1088b00020079800be0090002e009000008050001d
:1088c0000000e000e7ff3c007e0090008040eb00ed
:1088d00001487800210037003e019000220f9800e7
:1088e000140037002e0090001e00400090417800d8
:1088f000635798002e0090001e004000be009000bc
:108900009e80400091407800014878003e00900031
:108910001e004000ee509000014878003e0090009c
:108920000000e900300798002e0090000000e800e9
:1089300020079800be0090002e009000008050009c
:108940000000e000e7ff3c002e0890000000e80077
:108950001e0040008040eb00014878001e007800b7
:108960000080fa00000006000c00fa005007980092
:1089700010002000400798006800470012c0b300b4
:10898000800078005e00900049e80700100798001a
:108990001e0090000000e00002003a0000c0eb0062
:1089a000ad0037001e00900044e70700304188000a
:1089b000414188003041800041418000e00f50007b
:1089c000e08f58001a003a005e009000c1c5b30065
:1089d000415898000040eb00004f78000600370037
:1089e0001e80fb00de0090000080400001c2b3004a
:1089f000415898001e4fe8001e407800ea4f500092
:108a0000f7ff360000418000114180005e019000b8
:108a100070119800011998000041800011418000f8
:108a20005e01900010199800211998008900370004
:108a300032418000434180002207980033079800ac
:108a400030418000414180005e019000701198002b
:108a50000119980030418000414180005e01900082
:108a600010199800211998006800470012c0b3003f
:108a7000800078005e0090000de807001007980065
:108a80001e0090000000e00002003a0000c0eb0071
:108a9000710037001e00900008e707003041880091
:108aa000414188003041800041418000e00f50008a
:108ab000e08f580006003a0000418000114180001c
:108ac0005e019000701198000119980005003700b0
:108ad00030418000414180005e019000701198009b
:108ae000011998005e0090008018900070109000ae
:108af0005e01900010199800211998000000eb0009
:108b0000400798006800470012c0b300800078005a
:108b10005e009000e6e70700100798001e00900036
:108b20000000e00002003a0000c0eb004a003700fd
:108b30001e009000e1e607003041880041418800b6
:108b400012003700680047000041eb008000780009
:108b50005e009000d6e70700100798001e00900006
:108b60000000e00002003a0000c0eb003a003700cd
:108b70004e0090000000e800400798001e009000a2
:108b8000cee6070030418800414188003241800034
:108b9000434180002e009000be009000800f5100e5
:108ba000818f5900e7ff3a00324180004341800045
:108bb0002e009000be009000800f5100818f590060
:108bc0000c003a001e00900010407800fb4f40005f
:108bd000dcff32001e00900030489000e84f50004b
:108be000d8ff32001e00900030489000ef4f500038
:108bf000d4ff32000040eb00004f7800080037003f
:108c00001e80fb009e80fb001e019000e2c07800e9
:108c10005e01900000004100415898001e4fe8009e
:108c20001e407800ea4f5000f5ff36005e009000cd
:108c30002e019000be019000721098000318980059
:108c40005e0090002e019000be0190001218980066
:108c5000231898000040eb000080fa000000060096
:108c60000200fa00000f78000001eb009e0078007f
:108c70000040eb00020007000080fa000000060040
:108c80001a00fa0040579800310f9800420f9800e0
:108c9000be0890001107980060ce200020079800c1
:108ca0002468ef00aa1207000004e000050032006b
:108cb00080c1b30024e8b7000080eb006a013700f0
:108cc000000000000040eb00004f78000400370077
:108cd0001e0090000000e800100798001e4fe800fa
:108ce0001e009000104078000004e0000a003200ee
:108cf0001e00900090407800e0c2b30080cf50008a
:108d0000050032001e00900090407800c0c5b300fe
:108d100080cf5000eeff3a001e407800e84f500030
:108d200004003600f0c1b30024e8b7000080eb0077
:108d30004d0137001e00900090407800e0c2b30063
:108d400080cf50001e003a001e0090000000e80096
:108d5000100798000040eb00004f78000400370037
:108d60001e0090000000e800100798001e4fe80069
:108d70001e009000104078000004e0000500320062
:108d80001e00900090407800c0c5b30080cf500016
:108d9000f3ff3a001e407800e34f50000a0036000f
:108da000f0c1b30024e8b7000080eb002e013700cb
:108db0001e0090000000e800100798000300370034
:108dc0000000000001003700000000001e009000bd
:108dd00090407800c0c5b30080cf5000f4ff32004f
:108de0001e009000104078000004e000b4ff3a003c
:108df000be08900011079800a04180008000780014
:108e00002e009000beef07000300370000000000b6
:108e100001003700000000001e00900010407800a4
:108e2000004f7800e0c2b3009e40780080cf500031
:108e30004d003a001e0090000000e8001007980066
:108e40001e00900010407800004f7800e0c2b30090
:108e50009e40780080cf50000b0032001e4078000a
:108e60000004e00008003200c0c5b3009e40780056
:108e700080cf500004003200f0c1b30024e8b700f6
:108e80000080eb00f8003700e0c2b3009e4078009d
:108e900080cf500026003a00a04180007011900061
:108ea000801990000041800011418000800f510026
:108eb000818f590004003a00f0c1b30024e8b700e4
:108ec0000080eb00e80037001e0090000000e80082
:108ed000100798001e00900010407800004f7800a6
:108ee000c0c5b3009e40780080cf5000070032001c
:108ef0001e4078000004e00004003200f0c1b3001e
:108f000024e8b7000080eb00d7003700c0582800e5
:108f1000edfa0700060037001e0090000000e80090
:108f2000100798001e00900010407800004f780055
:108f3000c0c5b3009e40780080cf5000f6ff3200dd
:108f40001e4078000004e000b0ff3a00a04180001d
:108f5000ae0090006aef0700f0c1b30024e8b7004c
:108f60000080eb00c0003700c0c5b3009e40780011
:108f700080cf500034003a00a241800000418000c0
:108f8000114180007011980001199800a2418000e1
:108f900000418000114180001019980021199800ab
:108fa000a0418000c1c5b3004158980010c0b30073
:108fb000004f780006003700a14180001e80fb00b2
:108fc0000080400001c2b300415898001e4fe800e5
:108fd0001e407800ea4f5000f7ff36001e00900058
:108fe0000000e800100798001e0090001040780074
:108ff000004f7800c0c5b3009e40780080cf50007d
:1090000007003a00a0418000ae0090003cef07004e
:10901000f0c1b30024e8b7000080eb0092003700f5
:109020001e4078000004e0007aff3a00a041800072
:10903000ae00900032ef0700f0c1b30024e8b700a3
:109040000080eb00880037000040eb0020579800bc
:10905000030037000000000001003700000000009e
:109060001e00900010407800004f78000040eb0098
:10907000104798000e0037001e4090000080fb0053
:109080009e40780000004700614098001e4090001c
:109090000040e800104798001e0090000000e80023
:1090a000100798001e00900010407800004f7800d4
:1090b0001e4078000004e00007003200c0c5b30085
:1090c0009e40780080cf5000030032001e40900088
:1090d000eb4f5000e8ff36001e4090000080fb0080
:1090e000000047008040eb0061409800ee40900097
:1090f000e0c2b30080cf50001c003a007e409000d8
:109100000004e0000b003200fe409000e0c2b3001b
:1091100080cf500007003200a0418000ae009000d8
:10912000f7ee0700f0c1b30024e8b7000080eb00c1
:109130004d003700fe409000e0c2b30080cf5000e9
:109140000a003a000e4890000004e00007003200d8
:10915000a0418000ae009000e9ee0700f0c1b3002e
:1091600024e8b7000080eb003f00370066004700ae
:1091700055fa07000000e0000b00320066004700cf
:109180003b0007000000e00013003200170037002a
:109190001e0090000000e800100798001e009000dc
:1091a00010407800004f7800c0c5b3009e407800a2
:1091b00080cf5000f6ff32001e4078000004e0002f
:1091c000a4ff3a00a0418000ae009000ccee070062
:1091d0000000eb0024003700a0418000ae009000aa
:1091e000c7ee07000080eb001f0037006600470055
:1091f00035fa07000000e0000e003200a0418000b8
:10920000ae009000beee0700b0c1b30024e8b70086
:109210000080eb00140037001e0090000000e80002
:10922000100798001e00900010407800004f780052
:1092300001003700000000001e0090009040780000
:10924000c0c5b30080cf5000f3ff32001e4078004d
:109250000004e00081ff3a00a0418000ae009000d1
:10926000a7ee07000000eb000080fa0000000600f7
:109270001200fa00000f9800c0d1200030079800bb
:109280000000eb00700798000040eb00404798009a
:109290000c0037004e4090000080fb00ce40900054
:1092a0008180fb000e09900081004100114178008f
:1092b000c1da2000827078004e4090000040e80043
:1092c000404798004e409000eb4f5000f1ff3600b1
:1092d0008040eb00c0da200065f307000004e000e6
:1092e00004003a0020c1b30024e8b7000000eb00fe
:1092f000740037000040eb00404798000c00370036
:109300004e4090000080fb00ce4090008180fb002a
:10931000c2da2000e2c078003e0190000000410067
:10932000415898004e4090000040e80040479800a7
:109330004e409000ea4f5000f1ff3600a0418000ff
:1093400080189000701090003e01900070119800fd
:1093500001199800a0418000a018900010189000fa
:109360003e01900010199800211998003e019000cc
:109370006000b80010019800210198003e019000a3
:109380006000b8003001980041019800a0418000c1
:10939000900078003e009000010878006e004700c1
:1093a00022c1b300800078003e009000dce6070098
:1093b0000000e000020032000000eb004100370036
:1093c00018c8bf000004e0000d0032003e0090000d
:1093d0001000780011c0b3006022b8006011b8001e
:1093e00091f70700e00f5000e08f580004003200b2
:1093f00090c0b30024e8b7000000eb003100370054
:109400003e00900070119000801990000041800093
:1094100011418000800f5100818f590003003a00f4
:109420006000b800008fbe00040037003e009000ce
:109430007011900080199000028fbe003e009000d5
:1094400080189000701090003e0190001019980054
:10945000211998006e00470012c0b3008000780008
:109460003e00900092e50700400798004e009000f3
:109470000000e00004003a00b0c1b30024e8b700e7
:109480000000eb000f0037004e0090008be4070057
:1094900050079800610798003e0090001000780087
:1094a0001e02be005e019000ee0190000700070062
:1094b0000004e0000200320010002000010037002c
:1094c0000000eb000080fa00000006003400fa0003
:1094d000501798006217980073179800041f98009f
:1094e000151f98006a004700100798001a28ef001f
:1094f00000022000200798005e1090009080fb0082
:10950000104090000080fb004800dd0000807000eb
:10951000022020008000eb0026dc0700e0c2b30040
:10952000204f980010002000000f78000500370041
:109530006a0047001e00400001c2b30001487800e5
:109540001e0fe8001e007800ea0f5000f8ff3600fa
:1095500000c1b300505798000040eb0060579800de
:109560006e109000201798006e119000fe11900070
:1095700000002000f1ff20000202780003017800c3
:1095800080017800010078000302620000006100a1
:109590008000eb00c000dd00000020000001be00e4
:1095a0006120b80000017100818171004018de0067
:1095b0000100200000007800700f98006000b800e3
:1095c000301798004117980020cbb30070579800cf
:1095d00080272700400f9800002b2300500f980091
:1095e0000000eb00600f98000000eb0000179800ef
:1095f0000000eb00101798000000eb00000f78004f
:109600000c0037005e1090009080fb00104090002e
:109610000080fb004800dd00008070001e0040005c
:109620009e0090009e8040009140780001487800a4
:109630001e0fe8002e0090009e007800808f5000e2
:10964000f0ff3900e0c2b300304f98000e189000d0
:10965000201798000e1990009e199000000020001d
:10966000f1ff2000020278000301780080017800f9
:109670000100780003026200000061008000eb003e
:10968000c000dd00000020000001be006120b80025
:1096900000017100818171004018de00010020008e
:1096a00000007800700f98000000eb00000f7800b9
:1096b0000f0037005e1090009080fb00104090007b
:1096c0000080fb004800dd00008070008000780012
:1096d0002e0090001e004000008040009e00900080
:1096e0009e80400091407800014878001e0fe800fd
:1096f0002e0090009e007800808f5000edff390012
:109700006e119000fe1190005e1090007bee07003d
:1097100030079800410798005e1090009080fb0091
:10972000104090000080fb004800dd0000807000c9
:109730008041eb00000178003e009000ce009000d8
:10974000850f07000004e00004003a0090c0b30059
:1097500024e8b7000040eb000100370010c0b30060
:109760000080fa00000006000400fa00000f7800f4
:1097700021479800ae4190000001eb009e00780068
:109780000040eb00020007000080fa000000060025
:109790002400fa00405f9800710f980002179800ab
:1097a0002367980060ce200030079800c0d12000c9
:1097b000400798000000eb00500798006e0047003b
:1097c00002022200030222000288be006400400060
:1097d00002022200030222000288be006400400050
:1097e00002022200030220000288be006400400042
:1097f0008040eb00014878002468ef00a041800021
:10980000800078003e0090003ded07007e0890004b
:10981000adf807000000e00004003200c0c0b30053
:1098200024e8b7000080eb0036023700a04180003a
:10983000701190008019900000418000114180005b
:10984000800f5100818f590009003200a041800033
:1098500070119000801990003e00900080189000d8
:1098600070109000800f5100818f590007003a005e
:10987000a0418000be00900021ed0700f0c1b300c0
:1098800024e8b7000080eb001e0237005e00900065
:109890000000e80050079800a0418000ea0047005f
:1098a00012c0b30082e40700000f78001e007800a9
:1098b0000000e00007003a00a0418000be009000d8
:1098c0000fed0700b0c1b30024e8b7000080eb0043
:1098d0000c0237005e0090000000e800500798007e
:1098e000a0418000ea0047000041eb0070e407005f
:1098f000000f78001e0078000000e00007003a002a
:10990000a0418000be009000fdec0700b0c1b30094
:1099100024e8b7000080eb00fa0137002e609000c9
:109920000004e00023003a001d0037001e0078000c
:1099300010407800fb4f400007003200a04180003b
:10994000be009000eeec070060c1b30024e8b70051
:109950000080eb00eb0137005e0090000000e800a3
:1099600050079800a0418000ea0047000041eb004a
:109970004fe40700000f78001e0078000000e000b0
:1099800007003a00a0418000be009000dcec070018
:10999000b0c1b30024e8b7000080eb00d901370064
:1099a0001e007800104078000004e000dfff3a005d
:1099b0009a0137002a68ef000000eb0010079800ba
:1099c000930137001e007800104078000004e0008a
:1099d000e00032001e00780010407800fb4f40008d
:1099e000ba0032001e00780030489000e84f500066
:1099f000b60032001e00780030489000ef4f500053
:109a0000b20032001e007800304890000080fb0059
:109a1000700060000000e0006a0032001e0090004c
:109a20000000e800100798000040eb004047980055
:109a30000b0037004e4090000080fb00ce409000ad
:109a40008180fb001e017800e2c078000000470022
:109a5000614898004e4090000040e8004047980060
:109a60004e409000e74f500007003e004e409000ef
:109a70000080fb009e007800e140780000c2b30047
:109a800080cf5000ebff3a001e0078008048900025
:109a900000c2b30080cf5000250032004e4090003d
:109aa0000080fb0000004700e1c2b300614898005d
:109ab0004e4090000040e800404798000040eb0016
:109ac000504798000f0037004e4090000080fb0088
:109ad000de4090008180fb00e88040001e0178009d
:109ae000e2c0780000004700614898004e409000b6
:109af0000040e800404798005e4090000040e800c9
:109b0000504798005e409000e24f500008003e0031
:109b10005e4090000080fb00680040009e007800de
:109b2000e140780000c2b30080cf5000e6ff3a0069
:109b30004e4090000080fb00000047008040eb009a
:109b4000614898006e004700dff707000000e00062
:109b500007003200a0418000be00900068ec0700c2
:109b6000c0c0b30024e8b7000080eb0065013700f7
:109b7000a041800070119000801990003e0090007c
:109b80008018900070109000800f5100818f590054
:109b900007003a00a0418000be00900058ec07008a
:109ba000f0c1b30024e8b7000080eb005501370096
:109bb000200020005007980010c0b3002be8b70029
:109bc000450037006e004700c20020008000eb0017
:109bd00078da07000040eb00404798000c0037009f
:109be0004e4090000080fb00ce4090008180fb0042
:109bf0001e017800e2c078004e0190000000410094
:109c0000415898004e4090000040e80040479800be
:109c10004e409000ea4f5000f1ff36004e00900099
:109c200081d8200001087800de0090004e009000ee
:109c300041109800a04180008018900070109000a2
:109c40004e0190007011980001199800a041800009
:109c5000a0189000101890004e0190001019980064
:109c6000211998004e0190006000b8001001980082
:109c7000210198004e0190006000b800300198006a
:109c8000410198006a00470012c0b30080007800cc
:109c90004e009000b7e807000000e0000700320027
:109ca000a0418000be00900015ec070010c0b3007a
:109cb00024e8b7000080eb00120137005e0090003e
:109cc0000000e80050079800030037005e00900095
:109cd0000000e800500798002bc8bf000004e00017
:109ce0000d0032002b68ef00a2418000a0418000ef
:109cf0008018900070109000101998002119980099
:109d0000a0418000ea00470012c0b30068e30700ea
:109d1000000f780005003700a0418000ea004700ee
:109d20000041eb0062e30700000f78001e0078009e
:109d30000000e000b6003a00a0418000be009000a4
:109d4000efeb0700b0c1b30024e8b7000080eb00e0
:109d5000ec0037001e0090000000e000aa00320076
:109d60000000eb0060079800a2418000a041800045
:109d70008018900070109000101998002119980018
:109d8000a0418000ec00470012c0b30048e3070088
:109d9000000f78001e0078000000e00007003a0085
:109da000a0418000be009000d5eb0700b0c1b30019
:109db00024e8b7000080eb00d20037001e007800d6
:109dc0003ee207000000780060079800c0582800b5
:109dd0003df707000000e00007003200a0418000ce
:109de000be009000c6eb0700c0c0b30024e8b70077
:109df0000080eb00c30037002000200050079800cf
:109e0000a2418000a0418000801890007010900056
:109e10001019980021199800a0418000ea0047001d
:109e200012c0b30022e30700000f78001e00780084
:109e30000000e00007003a00a0418000be00900052
:109e4000afeb0700b0c1b30024e8b7000080eb001f
:109e5000ac0037001e00780018e20700304188008f
:109e600041418800160037005e0090000000e800c5
:109e700050079800a0418000ea0047000041eb0035
:109e80000be30700000f78001e0078000000e000e0
:109e900007003a00a0418000be00900098eb070048
:109ea000b0c1b30024e8b7000080eb009500370094
:109eb0001e00780001e2070030418800414188001f
:109ec0006e0090006101b800304180004141800087
:109ed000800f5100818f5900e3ff3a006e0090001f
:109ee0006101b8003041800041418000800f510085
:109ef000818f590008003a001e0078001040780059
:109f0000fb4f4000d8ff32001e0078003048900020
:109f1000e84f5000d4ff32006e004700c20020001e
:109f20008000eb00a3d907000040eb0040479800f9
:109f30000b0037004e4090000080fb00ce409000a8
:109f40008180fb001e017800e2c07800000047001d
:109f5000614898004e4090000040e800404798005b
:109f60004e409000ea4f5000f2ff36006e0047006e
:109f7000660007000000e00007003200a0418000fa
:109f8000be0090005eeb070010c0b30024e8b700ed
:109f90000080eb005b0037005e0090000000e800ee
:109fa00050079800a2418000a041800080189000d6
:109fb000701090001019980021199800a04180009d
:109fc000ea00470012c0b300b9e20700000f7800b2
:109fd0001e0078000000e00007003a00a041800069
:109fe000be00900046eb0700b0c1b30024e8b70004
:109ff0000080eb00430037001e0090000000e900e5
:10a00000100798000200370010c0b3002ae8b7001c
:10a010002ac8bf000004e0006afe32006e0047005c
:10a02000c100200079f807000000e00005003a00b8
:10a03000a0418000be00900031eb07000080eb00e3
:10a04000300037006e004700c20020008000eb00a7
:10a0500058d907000040eb00404798000c0037003b
:10a060004e4090000080fb00a2418000ce40900056
:10a070008180fb00fc804000e2c0780000004700c7
:10a08000614898004e4090000040e800404798002a
:10a090004e409000ea4f5000f1ff3600c0582800b3
:10a0a00089f607000000e00007003200a0418000b0
:10a0b000be00900012eb0700c0c0b30024e8b70058
:10a0c0000080eb000f0037006e0047000f00070014
:10a0d0000000e00007003200a0418000be009000b8
:10a0e00007eb070010c0b30024e8b7000080eb00c6
:10a0f00004003700a0418000be00900000eb070084
:10a100000000eb000080fa00000006003c00fa00ae
:10a11000501f98008e0d07000004e000020032007e
:10a120000080eb0037003700a14180006400470049
:10a13000f3ea07000040eb00004f78000900370009
:10a14000a24180001e80fb009e80fb00de19900073
:10a150008180410091407800000041004158980002
:10a160001e4fe8001e407800ea4f5000f4ff360012
:10a17000a041800080007800c0d12000e0ea070004
:10a18000a04180008041eb0012c0b300c1d120008b
:10a19000b4da0700100798001e0090000000e000ed
:10a1a00005003200a0418000e4004700d4ea070027
:10a1b0000080eb0013003700a041800081022000e6
:10a1c00080804000a041800012c0b30069e7070012
:10a1d000100798001e0090000000e00005003a0003
:10a1e000a0418000e4004700c5ea07000000eb0042
:10a1f00004003700a0418000e4004700c0ea0700e7
:10a200000080eb000080fa00000006004400fa0025
:10a21000701f9800012798001227980066004700d9
:10a22000100798002468ef001e0090007c0040009a
:10a2300012c0b300800078007e1890000cef070079
:10a240000004e00004003a0020c1b30024e8b70095
:10a250000080eb00f70037001e2090008040eb00ec
:10a26000216898000040eb00104798000d0037006f
:10a270001e4090000080fb009e4090008180fb000b
:10a280007e19900081004100914078001e219000cd
:10a2900000004100015898001e4090000040e80076
:10a2a000104798001e409000eb4f500007003e0002
:10a2b0001e4090000080fb00fe18900000804000cf
:10a2c000104078000004e000e9ff3a001e409000d2
:10a2d0000080fb009e209000008040008040eb004a
:10a2e000015898000e209000804078001e209000b9
:10a2f00051609800a041800080189000701090007c
:10a300001e21900030119800411198001e0090000d
:10a3100081d82000010878001e0190006000b8007c
:10a3200010019800210198001e0190006000b80003
:10a3300030019800410198001e0090008000eb0061
:10a34000411098001e0090008e209000611098002f
:10a35000a041800080189000701090001e019000b5
:10a360007011980001199800a0418000a018900079
:10a37000101890001e0190001019980021199800e3
:10a380009e009000c0d120005dea070013c0b3001a
:10a3900012c0b300c1d120001e00900031da0700c6
:10a3a000200798002e0090000000e000040032001a
:10a3b000b0c0b30024e8b7000080eb009d00370078
:10a3c0001e00900040109000601f9800c003200005
:10a3d0000e00400022c7b300800078001e009000ed
:10a3e00019db0700200798002e0090000000e00015
:10a3f0008d003a001e00900060109000e80f5000a1
:10a40000510032000040eb00104798000040eb0084
:10a41000004f78000c0037001e4090000080fb00c9
:10a420009e80fb001e019000fc80400062c178000d
:10a430009e209000827078001e4090000040e8004e
:10a44000104798001e4fe8001e407800e74f50006c
:10a4500007003e001e80fb009e0090007c00400034
:10a46000e140780000c2b30080cf5000eaff3a001c
:10a470001e009000c060900000c2b30080cf50006a
:10a480000a003a001e009000d060900000c2b300a5
:10a4900080cf500005003a001e009000e060900060
:10a4a00000c2b30080cf5000080032001e40900070
:10a4b0000080fb009e209000e2c2b3008270780012
:10a4c0001e4090000040e8001047980080c0b30094
:10a4d000004f78000c0037001e4090000080fb0009
:10a4e0009e80fb001e019000fc80400062c178004d
:10a4f0009e209000827078001e4090000040e8008e
:10a50000104798001e4fe8001e407800ea4f5000a8
:10a5100007003e001e80fb009e0090007c00400073
:10a52000e140780000c2b30080cf5000eaff3a005b
:10a530001e4090000080fb009e2090000041eb0038
:10a5400082707800170037000040eb001047980039
:10a550000c0037001e4090000080fb009e409000e1
:10a560008180fb001e019000fc80400062c17800e9
:10a570009e209000827078001e4090000040e8000d
:10a58000104798001e409000ea4f5000f1ff36003f
:10a590001e4090000080fb009e2090000041eb00d8
:10a5a000827078001e00900060109000804078005b
:10a5b0001e209000514898001e009000a0089000b6
:10a5c000100890001e219000700198000109980069
:10a5d0001e009000500890008000eb00c001dd00dc
:10a5e000020020001e009000400890008000eb0058
:10a5f00002004000838048001e219000100998004e
:10a60000210998001e009000c01090001e209000ac
:10a61000310898001e20900011c0b30021689800f6
:10a620000000eb0003003700b0c1b30024e8b7001e
:10a630000080eb000080fa00000006003e00fa00f7
:10a64000601f980066004700100798002468ef001c
:10a650006e189000206890000004e00004003a00aa
:10a6600070c0b30024e8b7000080eb00cc003700d6
:10a670006e18900030119000c0119000a041800031
:10a680008018900070109000800f5100818f590049
:10a6900004003200f0c1b30024e8b7000080eb00f2
:10a6a000bf0037001e009000fc0040006e189000b4
:10a6b0007800400012c0b300eded07000004e00098
:10a6c00004003a0020c1b30024e8b7000080eb008a
:10a6d000b30037001e00900081d8200001087800e8
:10a6e0001e0190006000b800100198002101980040
:10a6f0001e0190006000b8003001980041019800f0
:10a700006e189000300890008000e8001e00900055
:10a71000411098006e189000506090008080fb00ff
:10a720001e00900061109800a041800080189000e9
:10a73000701090001e01900070119800011998008f
:10a74000a0418000a0189000101890001e019000f9
:10a7500010199800211998009e009000c0d1200087
:10a7600067e9070013c0b30012c0b300c1d12000d5
:10a770001e0090003bd90700200798002e00900093
:10a780000000e00004003200b0c0b30024e8b700cd
:10a790000080eb00820037001e00900060109000e7
:10a7a000e80f50004f0032000040eb00004f7800ef
:10a7b0000040eb00104798000c0037001e80fb00a3
:10a7c0009e4090008180fb001e019000fc804000b4
:10a7d00062c17800ee189000827078001e4fe80089
:10a7e0001e4090000040e800104798001e40900076
:10a7f000e74f500008003e001e4090000080fb0024
:10a800009e0090007c004000e140780000c2b30050
:10a8100080cf5000e9ff3a001e009000c060900019
:10a8200000c2b30080cf50000a003a001e00900022
:10a83000d060900000c2b30080cf500005003a0005
:10a840001e009000e060900000c2b30080cf500076
:10a85000050032001e80fb00ee189000e2c2b3003b
:10a86000827078001e4fe80080c0b3001047980047
:10a870000c0037001e80fb009e4090008180fb0092
:10a880001e019000fc80400062c17800ee1890002c
:10a89000827078001e4fe8001e4090000040e800e3
:10a8a000104798001e409000ea4f500008003e00fc
:10a8b0001e4090000080fb009e0090007c00400045
:10a8c000e140780000c2b30080cf5000e9ff3a00b9
:10a8d0001e80fb00ee1890000041eb0082707800b3
:10a8e000120037000040eb00004f780008003700ee
:10a8f0001e80fb009e80fb001e019000fc8040003b
:10a9000062c17800ee189000827078001e4fe80057
:10a910001e407800ea4f5000f5ff36001e80fb0015
:10a92000ee1890000041eb00827078001e0090004d
:10a9300060109000804078006e1890005148980098
:10a940001e009000a0089000100890006e19900062
:10a9500070019800010998001e00900050089000b6
:10a960008000eb00c001dd00020020001e0090000e
:10a97000400890008000eb00020040008380480007
:10a980006e19900010099800210998001e0090008f
:10a99000c01090006e189000310898000000eb0085
:10a9a0000080fa00000006000200fa00000f7800a4
:10a9b000e642a9000a0037001e0078001040780027
:10a9c0000000fb000002b1001e0fe800200007009d
:10a9d000e082a800e082a9004001200006000700f4
:10a9e0001e007800104078000004e000f2ff3a00fa
:10a9f0000080fa00000006000600fa002007980018
:10aa00000000eb00000f78000b0037000000eb00a7
:10aa100010079800030037001e0090000000e800b7
:10aa2000100798009e0090002e009000808f50002c
:10aa3000f9ff35001e0fe800f0e124009e007800c9
:10aa4000808f5000f1ff34000080fa000000060003
:10aa5000561efa0041e52100810047008008780079
:10aa6000e4004700270f09008018eb0010002000c9
:10aa700001002000003f9800113f980010002000c6
:10aa800001002000203f9800313f98001000200076
:10aa900001002000403f9800513f98001000200026
:10aaa00001002000208798003187980010002000c6
:10aab00001002000009f9800119f980010002000c6
:10aac0000100200040a7980051a798001000200026
:10aad0000100200020af980031af98001000200046
:10aae0000100200040af980051af980010002000f6
:10aaf0000100200040bf980051bf980010002000c6
:10ab00000100200020079900310799001000200063
:10ab10000100200000179900111799001000200073
:10ab200001002000401799005117990010002000e3
:10ab300001002000001f9900111f99001000200043
:10ab400001002000401f9900511f990010002000b3
:10ab50000100200060279900712799001000200053
:10ab600001002000202f9900312f990010002000b3
:10ab700001002000602f9900712f99001000200023
:10ab800001002000003799001137990010002000c3
:10ab900001002000603799007137990010002000f3
:10aba00001002000003f9900113f99001000200093
:10abb00001002000403f9900513f99001000200003
:10abc00001002000008799001187990010002000e3
:10abd0000100200020879900318799001000200093
:10abe0000100200040879900518799001000200043
:10abf0000100200000979900119799001000200093
:10ac00000100200020979900319799001000200042
:10ac100001002000609799007197990010002000b2
:10ac200001002000009f9900119f99001000200052
:10ac300001002000609f9900719f99001000200082
:10ac40000100200020a7990031a7990010002000e2
:10ac50000100200040a7990051a799001000200092
:10ac60000100200000af990011af990010002000f2
:10ac70000100200020af990031af990010002000a2
:10ac80000100200040af990051af99001000200052
:10ac90000100200040b7990051b799001000200032
:10aca0000100200060b7990071b7990010002000e2
:10acb0000100200040bf990051bf99001000200002
:10acc0000100200060bf990071bf990010002000b2
:10acd00001002000400f9a00510f9a001000200040
:10ace00001002000600f9a00710f9a0010002000f0
:10acf0000100200000179a0011179a001000200090
:10ad00000100200020179a0031179a00100020003f
:10ad10000100200040379a0051379a0010002000af
:10ad200001002000408f9a00518f9a0010002000ef
:10ad300001002000209f9a00319f9a0010002000ff
:10ad40000100200000b79a0011b79a0010002000ff
:10ad50000100200060079b0071079b00100020008d
:10ad600001002000001f9b00111f9b00100020000d
:10ad700001002000201f9b00311f9b0010002000bd
:10ad800001002000401f9b00511f9b00100020006d
:10ad900001002000002f9b00112f9b0010002000bd
:10ada00001002000202f9b00312f9b00100020006d
:10adb00001002000402f9b00512f9b00100020001d
:10adc00001002000602f9b00712f9b0010002000cd
:10add0000100200000379b0011379b00100020006d
:10ade0000100200020879b0031879b00100020007d
:10adf0000100200000979b0011979b00100020008d
:10ae00000100200040979b0051979b0010002000fc
:10ae100001002000009f9b00119f9b00100020005c
:10ae20000100200020bf9b0031bf9b000044200098
:10ae30000001470010002000010020000089be0032
:10ae40000045200000014700100020000100200004
:10ae50000089be004048200000014700100020008b
:10ae6000010020000089be00c04b20000001470007
:10ae700010002000010020000089be00004c2000ce
:10ae80000001470010002000010020000089be00e2
:10ae9000004f2000000147001000200001002000aa
:10aea0000089be00805020000001470010002000f3
:10aeb000010020000089be00c050200000014700b2
:10aec00010002000010020000089be000051200079
:10aed0000001470010002000010020000089be0092
:10aee000c051200000014700100020000100200098
:10aef0000089be0000522000000147001000200021
:10af0000010020000089be0080522000000147009f
:10af100010002000010020000089be00c052200067
:10af20000001470010002000010020000089be0041
:10af300040532000000147001000200001002000c5
:10af40000089be004054200000014700100020008e
:10af5000010020000089be0080542000000147004d
:10af600010002000010020000089be0000572000d2
:10af70000001470010002000010020000089be00f1
:10af80008057200000014700100020000100200031
:10af90000089be004058200000014700100020003a
:10afa000010020000089be00805a200000014700f7
:10afb00010002000010020000089be00c05a2000bf
:10afc0000001470010002000010020000089be00a1
:10afd000c05b20000001470010002000010020009d
:10afe0000089be00805c20000001470010002000a6
:10aff000010020000089be00c05c20000001470065
:10b0000010002000010020000089be00005d20002b
:10b010000001470010002000010020000089be0050
:10b02000005e200000014700100020000100200009
:10b030000089be00405e2000000147001000200093
:10b04000010020000089be00c05f20000001470011
:10b0500010002000010020000089be00c060200018
:10b060000001470010002000010020000089be0000
:10b0700000612000000147001000200001002000b6
:10b080000089be0080612000000147001000200000
:10b09000010020000089be00c061200000014700bf
:10b0a00010002000010020000089be000062200086
:10b0b0000001470010002000010020000089be00b0
:10b0c0004063200000014700100020000100200024
:10b0d0000089be000066200000014700100020002b
:10b0e000010020000089be008066200000014700aa
:10b0f00010002000010020000089be000067200031
:10b100000001470010002000010020000089be005f
:10b11000006820000001470010002000010020000e
:10b120000089be0080682000000147001000200058
:10b13000010020000089be00c06920000001470016
:10b1400010002000010020000089be00c06a20001d
:10b150000001470010002000010020000089be000f
:10b16000006b2000000147001000200001002000bb
:10b170000089be00c06b20000001470010002000c5
:10b18000010020000089be00006c20000001470083
:10b1900010002000010020000089be00006d20008a
:10b1a0000001470010002000010020000089be00bf
:10b1b000406d200000014700100020000100200029
:10b1c0000089be00806d20000001470010002000b3
:10b1d000010020000089be00806e200000014700b1
:10b1e00010002000010020000089be00c06e200079
:10b1f0000001470010002000010020000089be006f
:10b20000c06f200000014700100020000100200056
:10b210000089be00007020000001470010002000df
:10b22000010020000089be000071200000014700dd
:10b2300010002000010020000089be0000722000e4
:10b240000001470010002000010020000089be001e
:10b250004072200000014700100020000100200083
:10b260000089be008072200000014700100020000d
:10b27000010020000089be00007520000001470089
:10b2800010002000010020000089be008075200011
:10b290000001470010002000010020000089be00ce
:10b2a000c0752000000147001000200001002000b0
:10b2b0000089be00407720000001470010002000f8
:10b2c000010020000089be008078200000014700b6
:10b2d00010002000010020000089be00c07820007e
:10b2e0000001470010002000010020000089be007e
:10b2f000c07920000001470010002000010020005c
:10b300000089be00007a20000001470010002000e4
:10b31000010020000089be00807a20000001470063
:10b3200010002000010020000089be00c07a20002b
:10b330000001470010002000010020000089be002d
:10b34000007b2000000147001000200001002000c9
:10b350000089be00007c2000000147001000200092
:10b36000010020000089be00407c20000001470051
:10b3700010002000010020000089be00807c200019
:10b380000001470010002000010020000089be00dd
:10b39000c07e2000000147001000200001002000b6
:10b3a0000089be00007f200000014700100020003f
:10b3b000010020000089be00807f200000014700be
:10b3c00010002000010020000089be00c07f200086
:10b3d0000001470010002000010020000089be008d
:10b3e0000080200000014700100020000100200024
:10b3f0000089be00008120000001470010002000ed
:10b40000010020000089be004081200000014700ab
:10b4100010002000010020000089be008081200073
:10b420000001470010002000010020000089be003c
:10b430004083200000014700100020000100200090
:10b440000089be0080852000000147001000200018
:10b45000010020000089be00008820000001470094
:10b4600010002000010020000089be00808a20001a
:10b470000001470010002000010020000089be00ec
:10b48000808d2000000147001000200001002000f6
:10b490000089be00408f20000001470010002000fe
:10b4a000010020000089be0000902000000147003c
:10b4b00010002000010020000089be00c091200083
:10b4c0000001470010002000010020000089be009c
:10b4d000c092200000014700100020000100200061
:10b4e0000089be00009420000001470010002000e9
:10b4f000010020000089be004095200000014700a7
:10b5000010002000010020000089be0000972000ec
:10b510000001470010002000010020000089be004b
:10b5200000992000000147001000200001002000c9
:10b530000089be00c09920000001470010002000d3
:10b54000010020000089be00409c2000000147004f
:10b5500010002000010020000089be00409d200056
:10b560000001470010002000010020000089be00fb
:10b57000809d2000000147001000200001002000f5
:10b580000089be00c09d200000014700100020007f
:10b59000010020000089be00009e2000000147003d
:10b5a00010002000010020000089be00409f200004
:10b5b0000001470010002000010020000089be00ab
:10b5c00080a02000000147001000200001002000a2
:10b5d0000089be00c0a0200000014700100020002c
:10b5e000010020000089be00c0a12000000147002a
:10b5f00010002000010020000089be00c0a2200031
:10b600000001470010002000010020000089be005a
:10b6100000a32000000147001000200001002000ce
:10b620000089be0040a32000000147001000200058
:10b63000010020000089be0040a420000001470056
:10b6400010002000010020000089be0080a420001e
:10b650000001470010002000010020000089be000a
:10b6600080a52000000147001000200001002000fc
:10b670000089be0000a72000000147001000200044
:10b68000010020000089be0080a7200000014700c3
:10b6900010002000010020000089be00c0a720008b
:10b6a0000001470010002000010020000089be00ba
:10b6b00000a8200000014700100020000100200029
:10b6c0000089be0000a920000001470010002000f2
:10b6d000010020000089be0040a9200000014700b1
:10b6e00010002000010020000089be0080a9200079
:10b6f0000001470010002000010020000089be006a
:10b70000c0aa200000014700100020000100200016
:10b710000089be0040ab200000014700100020005f
:10b72000010020000089be00c0ab200000014700de
:10b7300010002000010020000089be0000ac2000a5
:10b740000001470010002000010020000089be0019
:10b7500080ac200000014700100020000100200004
:10b760000089be00c0ac200000014700100020008e
:10b77000010020000089be0000ad2000000147004c
:10b7800010002000010020000089be0080ad2000d4
:10b790000001470010002000010020000089be00c9
:10b7a00040ae2000000147001000200001002000f2
:10b7b0000089be0080af200000014700100020007b
:10b7c000010020000089be00c0af2000000147003a
:10b7d00010002000010020000089be00c0b0200041
:10b7e0000001470010002000010020000089be0079
:10b7f000c0b120000001470010002000010020001f
:10b800000089be0040b32000000147001000200066
:10b81000010020000089be0080b320000001470025
:10b8200010002000010020000089be00c0b42000ec
:10b830000001470010002000010020000089be0028
:10b8400040b520000001470010002000010020004a
:10b850000089be00c0b52000000147001000200094
:10b86000010020000089be0000b620000001470052
:10b8700010002000010020000089be0080b62000da
:10b880000001470010002000010020000089be00d8
:10b89000c0b6200000014700100020000100200079
:10b8a0000089be0080b72000000147001000200082
:10b8b000010020000089be0040b8200000014700c0
:10b8c00010002000010020000089be0080b9200087
:10b8d0000001470010002000010020000089be0088
:10b8e000c0b9200000014700100020000100200026
:10b8f0000089be00c0ba20000001470010002000ef
:10b90000010020000089be00c0bb200000014700ec
:10b9100010002000010020000089be0000bd2000b2
:10b920000001470010002000010020000089be0037
:10b9300040bd200000014700100020000100200051
:10b940000089be0080bd20000001470010002000db
:10b95000010020000089be0080be200000014700d9
:10b9600010002000010020000089be00c0c020009f
:10b970000001470010002000010020000089be00e7
:10b9800000c220000001470010002000010020003c
:10b990000089be0040c220000001470010002000c6
:10b9a000010020000089be0080c220000001470085
:10b9b00010002000010020000089be0080c320008c
:10b9c0000001470010002000010020000089be0097
:10b9d000c0c320000001470010002000010020002b
:10b9e0000089be00c0c420000001470010002000f4
:10b9f000010020000089be0000c5200000014700b2
:10ba000010002000010020000089be00c0c52000f9
:10ba10000001470010002000010020000089be0046
:10ba200000c6200000014700100020000100200097
:10ba30000089be0040c72000000147001000200020
:10ba4000010020000089be0080c7200000014700df
:10ba500010002000010020000089be0080c82000e6
:10ba60000001470010002000010020000089be00f6
:10ba700000ca200000014700100020000100200043
:10ba80000089be0080ca200000014700100020008d
:10ba9000010020000089be0000cb2000000147000b
:10baa00010002000010020000089be0000cc200012
:10bab0000001470010002000010020000089be00a6
:10bac00080cc200000014700100020000100200071
:10bad0000089be00c0cd20000001470010002000fa
:10bae000010020000089be0040ce20000001470078
:10baf00010002000010020000089be00c0ce200000
:10bb00000001470010002000010020000089be0055
:10bb1000c0cf2000000147001000200001002000dd
:10bb20000089be0080d020000001470010002000e6
:10bb3000010020000089be0040d120000001470024
:10bb400010002000010020000089be0080d22000eb
:10bb50000001470010002000010020000089be0005
:10bb6000c0d220000001470010002000010020008a
:10bb70000089be00c0d32000000147001000200053
:10bb8000010020000089be0000d420000001470011
:10bb900010002000010020000089be0080d4200099
:10bba0000001470010002000010020000089be00b5
:10bbb00080d7200000014700100020000100200075
:10bbc0000089be0080d8200000014700100020003e
:10bbd000010020000089be0040da2000000147007b
:10bbe00010002000010020000089be0000db2000c2
:10bbf0000001470010002000010020000089be0065
:10bc000080db200000014700100020000100200020
:10bc10000089be0080dc20000001470010002000e9
:10bc2000010020000089be00c0dc200000014700a8
:10bc300010002000010020000089be00c0dd2000af
:10bc40000001470010002000010020000089be0014
:10bc500080e02000000147001000200001002000cb
:10bc60000089be0080e12000000147001000200094
:10bc7000010020000089be0000e320000001470011
:10bc800010002000010020000089be0080e3200099
:10bc90000001470010002000010020000089be00c4
:10bca00040e42000000147001000200001002000b7
:10bcb0000089be00c0e42000000147001000200001
:10bcc000010020000089be0080e52000000147003f
:10bcd00010002000010020000089be0080e6200046
:10bce0000001470010002000010020000089be0074
:10bcf00080e7200000014700100020000100200024
:10bd00000089be0000e8200000014700100020006c
:10bd1000010020000089be0080e8200000014700eb
:10bd200010002000010020000089be00c0e92000b2
:10bd30000001470010002000010020000089be0023
:10bd400080ea2000000147001000200001002000d0
:10bd50000089be0080eb2000000147001000200099
:10bd6000010020000089be00c0eb20000001470058
:10bd700010002000010020000089be00c0ec20005f
:10bd80000001470010002000010020000089be00d3
:10bd900000ed2000000147001000200001002000fd
:10bda0000089be0080ed2000000147001000200047
:10bdb000010020000089be00c0ed20000001470006
:10bdc00010002000010020000089be0040ef20008c
:10bdd0000001470010002000010020000089be0083
:10bde00080ef20000001470010002000010020002b
:10bdf0000089be0080f020000001470010002000f4
:10be0000010020000089be0080f2200000014700f0
:10be100010002000010020000089be00c0f22000b8
:10be20000001470010002000010020000089be0032
:10be300000f3200000014700100020000100200056
:10be40000089be0000f4200000014700100020001f
:10be5000010020000089be0040f4200000014700de
:10be600010002000010020000089be0080f42000a6
:10be70000001470010002000010020000089be00e2
:10be800080f5200000014700100020000100200084
:10be90000089be00c0f5200000014700100020000e
:10bea000010020000089be0080f62000000147004c
:10beb00010002000010020000089be00c0f6200014
:10bec0000001470010002000010020000089be0092
:10bed00000f72000000147001000200001002000b2
:10bee0000089be0080f720000001470010002000fc
:10bef000010020000089be00c0f7200000014700bb
:10bf000010002000010020000089be0040f9200040
:10bf10000001470010002000010020000089be0041
:10bf200080f92000000147001000200001002000df
:10bf30000089be0080fa20000001470010002000a8
:10bf4000010020000089be0080fb200000014700a6
:10bf500010002000010020000089be0080fc2000ad
:10bf60000001470010002000010020000089be00f1
:10bf7000c0fc20000001470010002000010020004c
:10bf80000089be0000fd20000001470010002000d5
:10bf9000010020000089be0000fe200000014700d3
:10bfa00010002000010020000089be0040fe20009b
:10bfb0000001470010002000010020000089be00a1
:10bfc00080fe20000001470010002000010020003a
:10bfd0000089be00c0ff20000001470010002000c3
:10bfe000010020000089be00c000210000014700c0
:10bff00010002000010020000089be000001210087
:10c000000001470010002000010020000089be0050
:10c01000c0012100000147001000200001002000a5
:10c020000089be000002210000014700100020002e
:10c03000010020000089be0000032100000147002c
:10c0400010002000010020000089be0040032100f4
:10c050000001470010002000010020000089be0000
:10c060008003210000014700100020000100200093
:10c070000089be004005210000014700100020009b
:10c08000010020000089be00c00621000001470019
:10c0900010002000010020000089be008007210060
:10c0a0000001470010002000010020000089be00b0
:10c0b000400821000001470010002000010020007e
:10c0c0000089be0080092100000147001000200007
:10c0d000010020000089be00c009210000014700c6
:10c0e00010002000010020000089be00c00a2100cd
:10c0f0000001470010002000010020000089be0060
:10c10000000b21000001470010002000010020006a
:10c110000089be00800b21000001470010002000b4
:10c12000010020000089be00800d210000014700b1
:10c1300010002000010020000089be00800e2100b8
:10c140000001470010002000010020000089be000f
:10c15000000f210000014700100020000100200016
:10c160000089be004011210000014700100020009e
:10c17000010020000089be0080122100000147005c
:10c1800010002000010020000089be008013210063
:10c190000001470010002000010020000089be00bf
:10c1a00000142100000147001000200001002000c1
:10c1b0000089be008014210000014700100020000b
:10c1c000010020000089be00001521000001470089
:10c1d00010002000010020000089be008015210011
:10c1e0000001470010002000010020000089be006f
:10c1f00080172100000147001000200001002000ee
:10c200000089be0000192100000147001000200035
:10c21000010020000089be008019210000014700b4
:10c2200010002000010020000089be00401b2100fa
:10c230000001470010002000010020000089be001e
:10c24000c01b210000014700100020000100200059
:10c250000089be00401e21000001470010002000a0
:10c26000010020000089be00801f2100000147005e
:10c2700010002000010020000089be0000202100e5
:10c280000001470010002000010020000089be00ce
:10c2900000212100000147001000200001002000c3
:10c2a0000089be008021210000014700100020000d
:10c2b000010020000089be00c022210000014700cb
:10c2c00010002000010020000089be000023210092
:10c2d0000001470010002000010020000089be007e
:10c2e000c0232100000147001000200001002000b1
:10c2f0000089be00c024210000014700100020007a
:10c30000010020000089be004025210000014700f7
:10c3100010002000010020000089be0040262100fe
:10c320000001470010002000010020000089be002d
:10c3300040282100000147001000200001002000db
:10c340000089be00c0282100000147001000200025
:10c35000010020000089be00c02921000001470023
:10c3600010002000010020000089be00802a21006a
:10c370000001470010002000010020000089be00dd
:10c38000802d210000014700100020000100200046
:10c390000089be00802f210000014700100020000e
:10c3a000010020000089be00c02f210000014700cd
:10c3b00010002000010020000089be00c0322100d2
:10c3c0000001470010002000010020000089be008d
:10c3d0000033210000014700100020000100200070
:10c3e0000089be00803321000001470010002000ba
:10c3f000010020000089be00c03321000001470079
:10c4000010002000010020000089be00003721003c
:10c410000001470010002000010020000089be003c
:10c42000803721000001470010002000010020009b
:10c430000089be00c03b2100000147001000200021
:10c44000010020000089be00c03c2100000147001f
:10c4500010002000010020000089be00c043210020
:10c460000001470010002000010020000089be00ec
:10c47000804521000001470010002000010020003d
:10c480000089be00c04521000001470010002000c7
:10c49000010020000089be00404621000001470045
:10c4a00010002000010020000089be00804621000d
:10c4b0000001470010002000010020000089be009c
:10c4c0000049210000014700100020000100200069
:10c4d0000089be00804a21000001470010002000b2
:10c4e000010020000089be00c04a21000001470071
:10c4f00010002000010020000089be00404b2100f8
:10c500000001470010002000010020000089be004b
:10c51000004e210000014700100020000100200013
:10c520000089be00804e210000014700100020005d
:10c53000010020000089be00804f2100000147005b
:10c5400010002000010020000089be00c04f210023
:10c550000001470010002000010020000089be00fb
:10c5600000532100000147001000200001002000be
:10c570000089be0080542100000147001000200007
:10c58000010020000089be00c054210000014700c6
:10c5900010002000010020000089be00405521004d
:10c5a0000001470010002000010020000089be00ab
:10c5b00080572100000147001000200001002000ea
:10c5c0000089be0000582100000147001000200033
:10c5d000010020000089be008059210000014700b1
:10c5e00010002000010020000089be00c059210079
:10c5f0000001470010002000010020000089be005b
:10c60000005a210000014700100020000100200016
:10c610000089be00c05a2100000147001000200020
:10c62000010020000089be00005d210000014700dc
:10c6300010002000010020000089be00405f2100a2
:10c640000001470010002000010020000089be000a
:10c65000c060210000014700100020000100200000
:10c660000089be0000612100000147001000200089
:10c67000010020000089be00806121000001470008
:10c6800010002000010020000089be00006221008f
:10c690000001470010002000010020000089be00ba
:10c6a000c0632100000147001000200001002000ad
:10c6b0000089be00406421000001470010002000f6
:10c6c000010020000089be008066210000014700b3
:10c6d00010002000010020000089be00006721003a
:10c6e0000001470010002000010020000089be006a
:10c6f00040672100000147001000200001002000d9
:10c700000089be0080672100000147001000200062
:10c71000010020000089be00806821000001470060
:10c7200010002000010020000089be0040692100a7
:10c730000001470010002000010020000089be0019
:10c74000006c2100000147001000200001002000c3
:10c750000089be00806c210000014700100020000d
:10c76000010020000089be00406e2100000147004a
:10c7700010002000010020000089be00807221000e
:10c780000001470010002000010020000089be00c9
:10c79000c0722100000147001000200001002000ad
:10c7a0000089be00407321000001470010002000f6
:10c7b000010020000089be008075210000014700b3
:10c7c00010002000010020000089be0040782100f8
:10c7d0000001470010002000010020000089be0079
:10c7e0008078210000014700100020000100200097
:10c7f0000089be00407a210000014700100020009f
:10c80000010020000089be00807a2100000147005d
:10c8100010002000010020000089be00407d2100a2
:10c820000001470010002000010020000089be0028
:10c83000807f21000001470010002000010020003f
:10c840000089be0080812100000147001000200007
:10c85000010020000089be00408221000001470045
:10c8600010002000010020000089be00008321008c
:10c870000001470010002000010020000089be00d8
:10c88000008421000001470010002000010020006a
:10c890000089be0000852100000147001000200033
:10c8a000010020000089be008086210000014700b1
:10c8b00010002000010020000089be0040872100f8
:10c8c0000001470010002000010020000089be0088
:10c8d000008a210000014700100020000100200014
:10c8e0000089be00808b210000014700100020005d
:10c8f000010020000089be00c08b2100000147001c
:10c9000010002000010020000089be00408c2100a2
:10c910000001470010002000010020000089be0037
:10c92000008f2100000147001000200001002000be
:10c930000089be0080902100000147001000200007
:10c94000010020000089be00809321000001470003
:10c9500010002000010020000089be00009421008a
:10c960000001470010002000010020000089be00e7
:10c970004094210000014700100020000100200029
:10c980000089be00809421000001470010002000b3
:10c99000010020000089be004096210000014700f0
:10c9a00010002000010020000089be0080982100b6
:10c9b0000001470010002000010020000089be0097
:10c9c0000099210000014700100020000100200014
:10c9d0000089be004099210000014700100020009e
:10c9e000010020000089be0080992100000147005d
:10c9f00010002000010020000089be00809a210064
:10ca00000001470010002000010020000089be0046
:10ca1000009e2100000147001000200001002000be
:10ca20000089be00c09f21000001470010002000c7
:10ca3000010020000089be0040a021000001470045
:10ca400010002000010020000089be0000a321008a
:10ca50000001470010002000010020000089be00f6
:10ca600040a3210000014700100020000100200029
:10ca70000089be0080a321000001470010002000b3
:10ca8000010020000089be0040a5210000014700f0
:10ca900010002000010020000089be0000a7210036
:10caa0000001470010002000010020000089be00a6
:10cab00080a7210000014700100020000100200095
:10cac0000089be0000a821000001470010002000de
:10cad000010020000089be0080a92100000147005c
:10cae00010002000010020000089be00c0a9210024
:10caf0000001470010002000010020000089be0056
:10cb000040aa210000014700100020000100200081
:10cb10000089be0080ae2100000147001000200007
:10cb2000010020000089be0000af21000001470085
:10cb300010002000010020000089be0080b3210009
:10cb40000001470010002000010020000089be0005
:10cb500000b4210000014700100020000100200067
:10cb60000089be0080b421000001470010002000b1
:10cb7000010020000089be0000b52100000147002f
:10cb800010002000010020000089be0000b9210033
:10cb90000001470010002000010020000089be00b5
:10cba00080b9210000014700100020000100200092
:10cbb0000089be0040bb210000014700100020009a
:10cbc000010020000089be00c0bb21000001470019
:10cbd00010002000010020000089be0040be21009e
:10cbe0000001470010002000010020000089be0065
:10cbf00040c021000001470010002000010020007b
:10cc00000089be00c0c021000001470010002000c4
:10cc1000010020000089be00c0c2210000014700c1
:10cc200010002000010020000089be0000c3210088
:10cc30000001470010002000010020000089be0014
:10cc400000c6210000014700100020000100200064
:10cc50000089be0040c821000001470010002000ec
:10cc6000010020000089be00c0c82100000147006b
:10cc700010002000010020000089be00c0c9210072
:10cc80000001470010002000010020000089be00c4
:10cc900080ca210000014700100020000100200090
:10cca0000089be0000cb21000001470010002000d9
:10ccb000010020000089be0080cc21000001470057
:10ccc00010002000010020000089be0080d021005b
:10ccd0000001470010002000010020000089be0074
:10cce000c0d22100000147001000200001002000f8
:10ccf0000089be0000d32100000147001000200081
:10cd0000010020000089be0080d3210000014700ff
:10cd100010002000010020000089be00c0d32100c7
:10cd20000001470010002000010020000089be0023
:10cd300000d4210000014700100020000100200065
:10cd40000089be0040d921000001470010002000ea
:10cd5000010020000089be00c0d921000001470069
:10cd600010002000010020000089be00c0dd21006d
:10cd70000001470010002000010020000089be00d3
:10cd800040df2100000147001000200001002000ca
:10cd90000089be0040e02100000147001000200093
:10cda000010020000089be0080e021000001470052
:10cdb00010002000010020000089be00c0e021001a
:10cdc0000001470010002000010020000089be0083
:10cdd00000e12100000147001000200001002000b8
:10cde0000089be0040e12100000147001000200042
:10cdf000010020000089be0080e121000001470001
:10ce000010002000010020000089be00c0e12100c8
:10ce10000001470010002000010020000089be0032
:10ce200000e2210000014700100020000100200066
:10ce30000089be0040e221000001470010002000f0
:10ce4000010020000089be0080e2210000014700af
:10ce500010002000010020000089be00c0e2210077
:10ce60000001470010002000010020000089be00e2
:10ce700000e3210000014700100020000100200015
:10ce80000089be0040e3210000014700100020009f
:10ce9000010020000089be0080e32100000147005e
:10cea00010002000010020000089be00c0e3210026
:10ceb0000001470010002000010020000089be0092
:10cec00000e42100000147001000200001002000c4
:10ced0000089be0040e4210000014700100020004e
:10cee000010020000089be0080e42100000147000d
:10cef00010002000010020000089be00c0e42100d5
:10cf00000001470010002000010020000089be0041
:10cf100000e5210000014700100020000100200072
:10cf20000089be000000eb001007980030012000cf
:10cf3000000f78001a00370040e52100000047008c
:10cf4000100078007400b900000078001e00400056
:10cf50004200dd00e4004700008040001000be00f9
:10cf6000100798001e0090000040780061406000ab
:10cf70000080fb00610060004200dd0012168000ae
:10cf8000b1ff2f00810061000100700010168800c1
:10cf9000c222a900c222a800c242a9001e0fe900b5
:10cfa0001e0078000000e000e3ff3d000080fa0072
:10cfb000000006000000fa007016800064006000a7
:10cfc00000f0a7000000ea000000e9004f00de00ca
:10cfd000004078000080fa00000006000000fa001f
:10cfe000d04180000080fa00000006000000fa0036
:10cff000b0418000c14180000080fa0000000600be
:10d000000000fa00ce22a800cc22a900cc42a80041
:10d01000cc62a8000080fa00000006000000fa00c0
:10d02000f5010700ce22a8000040eb000080fa00c6
:10d03000000006001800fa00881f78008a9fbe00d2
:10d040000004780021579800220f9800330f9800b1
:10d0500080002000000f7800ce22a9002e50900002
:10d060000080fb006600b90080007800604f280057
:10d070000080400010407800005798002e09900072
:10d08000be09900062079800730798002e50900028
:10d090000080fb006600b90080007800604f280027
:10d0a0000080400010409000204f98000e08900033
:10d0b0000060a000000f98000e509000d5010700fe
:10d0c0007e489000d30107006e489000d101070010
:10d0d0005e489000cf0107004e489000cd01070048
:10d0e0002e489000cb0107002e5090000080fb00de
:10d0f0006600b900000078008080e800604f2800da
:10d1000000804000100078000000e00014003200b1
:10d110002e5090000080fb006600b90000007800ef
:10d120008080e800604f28000080400010007800f8
:10d13000e10f50000a0032002e5090000080fb00ea
:10d140006600b900000078008080e800604f280089
:10d150000080400010007800e40f50000a003a0000
:10d16000c0010700404798001e0fe9004e409000a4
:10d17000e14f400014003a001e0078000000e0007b
:10d18000f7ff3a00110037002e5090000080fb009e
:10d190006600b900000078008080e800604f280039
:10d1a0000080400010007800e20f500007003a00b5
:10d1b000ac010700ab01070050479800a901070028
:10d1c0004047980001003700000000002e509000fa
:10d1d0000080fb006600b900000078008080e80055
:10d1e000604f28000080400010007800e10f5000e0
:10d1f00019003a000040eb00404798000040eb0067
:10d20000204798000e0037000080eb00000f7800e8
:10d2100094010700404798001e0fe9004e4090001f
:10d220000004e00003003a001e0078000000e00067
:10d23000f7ff3a002e4090000040e8002047980099
:10d240002e409000e14f4000030032004e4090001d
:10d250000004e000ecff32002e5090000080fb0044
:10d260006600b900000078008080e800604f280068
:10d270000080400010007800e40f500028003a00c1
:10d28000780107000080fb008000eb00c800dd0093
:10d290000000200030079800410798003e059000ec
:10d2a000ce0590006f0107000080fb008000eb00be
:10d2b000c000dd00000020000a0040008b80480014
:10d2c00030079800410798003e059000ce05900079
:10d2d000640107000081fb008001eb004818dd00bd
:10d2e000c810de00810070004810dd000a00400018
:10d2f0008b80480030079800410798003e05900059
:10d30000ce059000570107000080fb008000eb0075
:10d310000a0040008b8048003007980041079800c1
:10d3200000c0eb003b0107002e5090000080fb0086
:10d330006600b90000007800e4004000604f28005b
:10d3400000804000104078000004e00001003a0036
:10d35000ce22a8002e019000be019000028cbe00db
:10d36000ce01900023049800080078004f05be000d
:10d370004f0478000080fa00000006001e00fa004a
:10d38000100f9800210f9800320f980010c0b300c2
:10d39000404798003cc8bf000004e00009003a0084
:10d3a0001e099000ae0990004918dd00c710de008c
:10d3b000810070004910dd00300798004107980097
:10d3c000040037001e099000ae0990003207980053
:10d3d000430798006c0047003e019000ce0190008a
:10d3e00081c0b30013ff07004e4890000004e00026
:10d3f00010003200780047003e019000ce019000fe
:10d4000081c0b3000bff07004e099000de099000b9
:10d410006207980073079800ee099000030f9800c8
:10d420004e4890000004e000020032000040eb0093
:10d4300047003700f02f2000000f78000004200084
:10d4400010079800030037001e0090000000e9005c
:10d45000100798001e0090000000e000faff3a005c
:10d4600000010700204f98001e0fe9000004200073
:10d4700010079800030037001e0090000000e9002c
:10d48000100798001e0090000000e000faff3a002c
:10d490002e489000e14f400003003a001e00780043
:10d4a0000000e000eeff3a001e0078000000e000ff
:10d4b000030032002e489000e24f4000030032008b
:10d4c0000040eb00404798001d0037000000eb00d3
:10d4d000000f7800120037003e0890000000e000c6
:10d4e0000d003200f00f2000401388000000000003
:10d4f00000138000610060000000e000fcff3200cb
:10d500003e0890001e0040004113800081407800da
:10d510000148780001003700d20007001e0fe80024
:10d52000d04180009e007800808f5000eaff3900d3
:10d5300000c0eb00b700070000c0eb00b50007001b
:10d5400000c0eb00b3000700ce22a8004e409000c0
:10d550000080fa00000006001c00fa007007980026
:10d56000010f9800120f98004357980010c0b300a5
:10d57000604798007e0090008e089000e00f5000f9
:10d58000e08f580006003a004e5090000004e00082
:10d5900003003a000040eb00604798006900370044
:10d5a0003cc8bf000004e0000c003a007e0190007f
:10d5b0008e0990004918dd00c710de008100700060
:10d5c0004910dd00680247000001be00a1c0b300a1
:10d5d0000400780097fe07000b0037007600470034
:10d5e0007e0190008e099000a1c0b30091fe07005b
:10d5f0003e099000ce09900042079800530798001a
:10d60000de099000630798000e4890000004e000d7
:10d61000030032000040eb006047980048003700ec
:10d62000e0cfb3007b0007000000eb00000f7800a4
:10d630000d0037001e0890001e00400010407800ca
:10d640000080fb00401388000000000000138000f1
:10d65000610060000000e000fcff32004013800029
:10d66000704798001e0fe800d04180009e007800af
:10d67000808f5000efff390000c0eb00650007000d
:10d6800000c0eb00630007007600070070479800b9
:10d690007e4090000080fb006f006000e50f5000ae
:10d6a000030032000040eb00604798002200370082
:10d6b00040c728005100200010079800210798005b
:10d6c000f00f2000401388001e009000ae00900074
:10d6d00061005000e0805800100798002107980072
:10d6e0000000000000138000610060000000e00006
:10d6f000fcff320040138000704798007e4090008d
:10d700000004e00005003a001e009000ae0090000a
:10d71000e00f5000e08f5800e9ff3a001e00900033
:10d72000ae009000e00f5000e08f580002003a0079
:10d730000040eb006047980000c0eb003500070098
:10d74000ce22a8006e4090000080fa000000060083
:10d750000000fa00701680004300de0061406000a7
:10d760000080fa00000006000800fa0060479800f8
:10d77000ee409000014f780015003700b07c20008b
:10d780000100200010079800210798000000000009
:10d790009e0090002e0090000100700000f0a70095
:10d7a0000000ea000000ea004f00de0000417800bf
:10d7b0001e009000ae00900061005000e080580014
:10d7c00010079800210798000204e000f0ff3a00db
:10d7d0001e80fb000000ea004f00de0000407800e1
:10d7e0001e4fe9000004e000e4ff3a0000000000e2
:10d7f0000080fa00000006000000fa00011380001b
:10d80000f0ff270000806000001388000080fa000d
:10d81000000006000400fa00204798002e40900007
:10d820000080fb004013880000000000001380000f
:10d83000620060000000e000fcff3a000000000011
:10d8400000138000610060000000e000fcff320077
:10d8500040138000004f78000040eb000080fa0089
:10d86000000006000000fa00f00f200040138800be
:10d870000000000000138000610060000000e00074
:10d88000fcff320040138000004078000080fa0066
:10d89000000006000200fa00000f78006022ef008e
:10d8a0006222ef00101380001e0070001013880029
:10d8b00062c2a8006302a9006382a900e502a90070
:10d8c000e4e2a80061e2a8000080fa00000006007f
:10d8d0002c00fa00881f78003000200020079800f4
:10d8e00060e120008040eb000148780070e12000fa
:10d8f0008040eb00014878003628ef003828ef0020
:10d90000ce22a80000052000000f78001e0078003d
:10d910000000e00012003a00f0032000ddff0700e5
:10d920001e0037001e007800e80f5000100036007f
:10d930002e0090000000e900200798009e0078006b
:10d94000638060000000e000020032001e017800e9
:10d95000640f41001e0078004200de00000f7800d6
:10d960001e0078000000e000eeff3a0001003700e2
:10d97000000000001e0fe9001e0078004200dd00dc
:10d980000080ea00fc0060002e0090008100700022
:10d990000002200001007000beff070010c0b300ad
:10d9a00071ff07000000eb00000f78000300370054
:10d9b00000c0eb0097ff07001e0fe8001e00780074
:10d9c000e90f5000faff3600ce22a90010c0b300c4
:10d9d00065ff07006c0047006011b8008040eb0055
:10d9e00094fd07004e489000e14f400006003200d1
:10d9f0004e4890008080fb00700f20000080600087
:10da0000e10f500006003200ce22a80060e12000a5
:10da100021c0b3000148780060e120006a013700ae
:10da2000600220000e004000a21a20000300200027
:10da300021c0b3007ffd07003e119000ce11900081
:10da40006207980073079800de119000030f98009a
:10da50007e0190008e099000f0ff20000100200060
:10da6000020278000301780080017800010078004c
:10da700003026200000061008000eb00c000dd00d6
:10da8000000020000001be006120b800000171000c
:10da900081817100a01a200001002000800f510038
:10daa000818f590042003a006e00900064006000cf
:10dab0000000e0003e003a00f0ff2000000f780078
:10dac000600220000e00400002002000030024003d
:10dad00011c0b30057fd07003e119000ce11900019
:10dae0006207980073079800de119000030f9800fa
:10daf0001e0fe9004e4890000004e00003003200d1
:10db00001e0078000000e000edff3a0060022000f7
:10db10000e0040006011b80001c1b30045fd0700d0
:10db20003e119000ce119000620798007307980094
:10db3000de119000030f98007e0190008e09900086
:10db40000000200001002c00020278000301780090
:10db5000800178000100780003026200000061008b
:10db60008000eb00c000dd00000020000001be00ce
:10db70006120b80000017100818171000000200067
:10db800001002c00800f5100818f590006003a00df
:10db90004e4890000004e00003003a0010c0b300bb
:10dba0003ce8b700170037003c68ef00150037006d
:10dbb0003c68ef00f0ff2000000f780060022000ba
:10dbc0000e0040006011b80011c0b30019fd07003d
:10dbd0003e119000ce1190006207980073079800e4
:10dbe000de119000030f98001e0fe9004e489000d0
:10dbf0000004e000030032001e0078000000e00096
:10dc0000eeff3a001e0078000000e00005003a0038
:10dc100060e1200021c0b30001487800ce22a800b6
:10dc2000e800370020c0b300cffe0700e00320006b
:10dc300018ff0700f0ff2000000f780060022000ae
:10dc40000e0040006011b80031c0b300f9fc0700bd
:10dc50003e119000ce119000620798007307980063
:10dc6000de119000030f98001e0fe9004e4890004f
:10dc70000004e000030032001e0078000000e00015
:10dc8000eeff3a000040eb00304798000040eb0008
:10dc900020479800130037003e4090000084fb00ae
:10dca000f0fe070088004700a05098003e4090001a
:10dcb0000040e800304798002e4090000004e0004b
:10dcc00005003a002e509000e24f400002003a005a
:10dcd0000040eb00304798002e4090000040e800e4
:10dce000204798002e409000f34f5000eaff360086
:10dcf00000202000d0418800b07080000080a0008b
:10dd0000b0708800d0418000c07088002e50900014
:10dd10008080fb00000c2000008060000000e0001c
:10dd20002e0032001e5890000081fb008001eb00a5
:10dd3000f0032000010020000202780003017800b7
:10dd40008001780001007800030262000000610099
:10dd50008000eb00c000dd00000020000001be00dc
:10dd60006120b8000001710081817100c011dd00e7
:10dd7000020020002e5890000080fb004800dd00cb
:10dd80008000eb0000017100818171003e5890001d
:10dd90000080fb008000eb000000710081807100ba
:10dda00030079800410798003e009000ce00900098
:10ddb00061014000e08148004a18dd00c610de0025
:10ddc000810070004a10dd0061005000e0805800c2
:10ddd000b0418800c1418800610037000e589000b2
:10dde0000080fb008000eb00c001dd00020020008d
:10ddf0001e5890000080fb004800dd008000eb0012
:10de000000017100818171002e5890000080fb009c
:10de10008000eb00000071008180710030079800e5
:10de2000410798003e019000ce01900000fc2f00b9
:10de300031002000020278000301780080017800a0
:10de40000100780003026200000061008000eb0026
:10de5000c000dd00000020000001be006120b8000d
:10de6000000171008181710032079800430798001a
:10de70003e009000ce0090004a09dd004600de0022
:10de800000007100c608de003007980041079800c6
:10de90003e589000634060000040400080407800a1
:10dea0004e5890000080fb004700de0000407800e4
:10deb00000c07000204f98007e5090006f406000be
:10dec000304f98003e4890000080fb0069005000f1
:10ded000110020000008dd00304f98003e00900047
:10dee000ce00900061014000e08148002e48900083
:10def0000080fb000080e800110020000008dd0029
:10df00008000eb00009ab90004027800028bb9008f
:10df100086027800050242000010b80001024200ab
:10df2000840078003e4990000281fb008001eb00f4
:10df3000028ab90004027800009bb90086027800ca
:10df4000050242000200b80001024200840078008d
:10df500061005000e0805800b0418800c141880055
:10df6000600220000e0040006011b80011c1b30033
:10df700030fc07003e119000ce119000620798001f
:10df800073079800de119000030f9800d0418000c5
:10df90008000eb00640220000e0242000001be007f
:10dfa00071c0b3000400780022fc07003e1190000d
:10dfb000ce1190006207980073079800de11900060
:10dfc000030f980060e120004f0478000080fa0001
:10dfd000000006000000fa0010002000e2fd07002b
:10dfe000018220000040eb002e00070010002000fe
:10dff000ddfd07004196290030c0b300290007006d
:10e000000080fa00000006000000fa00c682a900a5
:10e01000c662a900c6a2a900c602a800ca82a800ba
:10e02000ca62a800caa2a900ce22a8000080fa00f5
:10e03000000006000000fa0001128000f0ff270037
:10e0400000806000001288000080fa0000000600d6
:10e050000400fa0020479800ca82a900300020007e
:10e06000430207002e4090000080fb0040020700a2
:10e070004e020700000f78001e0078004800dd0007
:10e08000000f7800490207001e0f7000ca82a80026
:10e0900010002000b4fd07001e0078000080fa0088
:10e0a000000006000400fa00004f780011079800f5
:10e0b000ca82a900200020002d0207001e80fb005c
:10e0c0002b0207001e0090004800de002802070017
:10e0d0009e009000f00f20000080600024020700e6
:10e0e000ca82a800100020009ffd07000080fa00ef
:10e0f000000006000200fa00004f7800ca62a90082
:10e10000300520001a020700f00e20001802070058
:10e11000e0062000160207001e80fb001402070024
:10e120000000eb00120207000000eb0010020700e5
:10e130000000eb000e0207000000eb000c020700dd
:10e14000ca62a8000080fa00000006000000fa0081
:10e15000ca62a900d004200005020700a00e20001a
:10e1600003020700d006200001020700400520003e
:10e17000ff0107000000eb00fd0107000000eb00bd
:10e18000fb0107000000eb00f90107000000eb00b5
:10e19000f7010700ca62a8006009200072fd0700ad
:10e1a0000080fa00000006000000fa008080eb000a
:10e1b000b0c0b300bbff07000080fa0000000600fb
:10e1c0000400fa00204798000000eb00000f7800e0
:10e1d000b0c0b3009eff0700000f7800ae40900073
:10e1e00010c3b30080cf500006003a001e00780034
:10e1f0000000e00008003200807f2f001e0f40006a
:10e20000050037001e007800e10f400002003200d8
:10e21000808020001e0f40009e007800b0c0b30038
:10e22000a0ff07000080fa00000006000600fa00c8
:10e230001007980021079800ca62a9000000eb00af
:10e24000000f7800080037001e0090001040780092
:10e250000080fb009e0090008100e80011079800fc
:10e26000c30107001e0fe8002e0090009e007800fa
:10e27000808f5000f4ff3500ca62a8000080fa00c9
:10e28000000006000000fa00caa2a900a0002000b9
:10e2900035fd0700caa2a8000080fa0000000600b1
:10e2a0000400fa0040c0b30069ff0700000f7800c7
:10e2b0009e007800c00320000001780011000900d2
:10e2c0008280d800204798009e007800c00320007c
:10e2d00000017800110009008280d8008000fd0054
:10e2e000304798002e4090008080fb00a000200066
:10e2f00000017800110009008280d80000407800f9
:10e3000002c3b30082404000c0e120000148780011
:10e310002e4090008080fb00a000200000017800cb
:10e32000110009008280d8008000fd0000407800c4
:10e3300002c3b30082404000d0e1200001487800d1
:10e34000e0e12000a1c3b300014878003e40900006
:10e350008080fb00a000200000017800110009006f
:10e360008280d8000040780002c3b30082404000a1
:10e37000f0e12000014878003e4090008080fb00e2
:10e38000a000200000017800110009008280d80060
:10e390008000fd000040780002c3b30082404000ce
:10e3a00000e22000014878000080fa00000006002a
:10e3b0000200fa00ca62a9000000eb00000f78001a
:10e3c0000800370000000000401680006100600077
:10e3d0000000e000fcff32000000eb0064010700d9
:10e3e0001e0fe800704120009e007800808f5000d2
:10e3f000f4ff3400ca62a8000080fa0000000600a2
:10e400000800fa0030079800e642a9000000eb007f
:10e41000000f7800140037001e0078004200dd0075
:10e42000be009000008040001000be001007980061
:10e430001e0078000000e8004200dd00be009000f1
:10e44000008040001000be0020079800ae00900041
:10e450001e0090001f000700c4c2a800c4c2a9008b
:10e460001e0fe8001e0fe8001e007800e90f5000a4
:10e47000e9ff34000080fa00000006000600fa0000
:10e48000200798000000eb00000f78000b00370019
:10e490000000eb0010079800030037001e009000fa
:10e4a0000000e800100798009e0090002e009000e9
:10e4b000808f5000f9ff35001e0fe800f0e12400c6
:10e4c0009e007800808f5000f1ff34000080fa0039
:10e4d00000000600e001fa0060af990071af9900fa
:10e4e000e4004700623328006f000900b21878008a
:10e4f000410e200081004700624128006f000900a2
:10e50000b21878008e007800411cb0000b000900a2
:10e510008018eb000000eb0010079800600020005e
:10e52000000f7800190037007ea891006700b9003d
:10e53000000078001e0040004200dd00410e200077
:10e540008e804000008040001000be001007980040
:10e550001e00900000407800614060000080fb00d9
:10e56000610060004300dd004217800071ff2f0052
:10e57000810061000100700040178800e2a2a9003c
:10e58000e2a2a800e862a9001e0fe9001e007800c0
:10e590000000e000e4ff3d0050002000000f780084
:10e5a000160037001e0078004200dd00411c2000ec
:10e5b0008e804000008040001000be0010079800d0
:10e5c0001e00900000407800614060000080fb0069
:10e5d000610060004300dd004217800071ff2f00e2
:10e5e000810061000100700040178800e2a2a900cc
:10e5f000e2a2a800e862a9001e0fe9001e00780050
:10e600000000e000e7ff3d0060002000000f780000
:10e61000180037006ea891006700b900000078006c
:10e620001e0040004200dd00e40047000080400082
:10e630001000be00100798001e00900000407800f7
:10e64000614060000080fb00610060004300dd006d
:10e650004217800071ff2f008100610001007000ef
:10e6600040178800e2a2a900e2a2a800e862a9007f
:10e670001e0fe9001e0078000000e000e5ff3d00ed
:10e680000080fa00000006002800fa00d30007000e
:10e690004156280013000900311f78008e02b10096
:10e6a0000e00780056ff0700ffff37000000fa0059
:10e6b0004382a9004362a9004342a9004322a90062
:10e6c0004302a80042e2a90042c2a90042a2a80057
:10e6d000101280000020a0000030a1000040a00027
:10e6e00010128800101280000000a0000010a0008e
:10e6f0001012880040c2a90041e2a80041a2a9006e
:10e700004022a9004002a9006382a9006362a90017
:10e710006342a9006322a9006302a80062e2a90083
:10e7200062c2a90062a2a800101380000020a0000d
:10e730000030a1000040a0001013880010138000da
:10e740000000a0000010a0001013880060c2a90003
:10e7500061e2a80061a2a9006022a9006002a900ec
:10e760000080fa00000006000000fa003ec8bf006a
:10e770000080fb0042dc20008000780000e12000e7
:10e78000a2ee070000408800004080000000e0008a
:10e790001f003a002156280040dc200017d7070050
:10e7a00010408800104080000000e00010003a0097
:10e7b000ffff370010408000800178000202200037
:10e7c0001100200000df20009ddc07000000000099
:10e7d00040168000610060000000e000fcff320095
:10e7e0000102200000df200090fe0700010037003a
:10e7f00000000000104080007fdc07000000e00007
:10e80000ecff320010408000ffd30700e8fe070055
:10e810000080fa00000006000000fa0060022000fc
:10e82000303a8800203a80000060a1000070a1000a
:10e83000203a8800213a800000fe2f00008060000e
:10e84000203a88004827ef0040a7a90012002000c6
:10e8500080072000a109200033742000804978003f
:10e86000814978008249780012002000600420006d
:10e8700071052000237420008049780081497800c8
:10e880008249780000000000113a80000000270053
:10e890008080600000002100808f5000faff3a0065
:10e8a00000000000113a800000022000008060009b
:10e8b0000000e000fbff32000080fa0000000600cc
:020000040000fa
:10e8c000100e000006000000020000002a2e6d005d
:10e8d00070330000c40d00004c0000000000000078
:10e8e0003e08000002000000020000002f000000af
:10e8f000000800001800000000000000400c0000ac
:10e9000084010000000000002c0800000a00000044
:10e9100002000000ffffff00ffffff00ffff5200ab
:10e920000d000000180800001400000000000000a6
:10e93000400800000002000000000000400a000043
:10e940000002000000000000160e0000060000009b
:10e950000000000036080000080000000000000071
:10e960001c0e000006000000000000000000000077
:020000040000fa
:10e970000400fa00204798002e4090000080fb0021
:10e98000401288000000000000128000610060005a
:10e990000000e000fcff320040128000004f7800d1
:10e9a0000040eb000080fa00000006000000fa00c2
:10e9b000f00f2000401288000000000000128000cc
:10e9c000610060000000e000fcff320040128000a7
:10e9d000004078000080fa00000006000000fa0005
:10e9e000100020006019880010002000601b8800c3
:10e9f00010002000501988006820ef006a20ef0006
:10ea0000de82a900c022a900c042a900e442a900f8
:10ea1000c0c2a900dea2a900e462a900c0e2a90068
:10ea2000c1a2a900c5a2a8000080fa00000006004b
:020000040000fa
:0200000401f009
:04000c00f8ff0000f9
:020000040000fa
:0200000401f009
:040010007fff00006e
:020000040000fa
:0200000401f009
:040014007fff00006a
:00000001FF
